:100000000C941E060C94EA280C9417290C944606AE
:100010000C9446060C9446060C9446060C94460630
:100020000C9446060C9446060C9422130C94460637
:100030000C9446060C9446060C9446060C94460610
:100040000C9444290C9446060C94322D0C94752D76
:100050000C9446060C9446060C9446060C944606F0
:100060000C9446060C9446062B198D196C196F19C1
:100070007219751978197B197E198D198719BF1A8C
:10008000C11AC11ABF1AC11AC11AC11AC11AC11A9A
:10009000C11AC11AC11AC11AC11AC11AC11AC11A88
:1000A000451AC11AC11AC11AC11AC11AB619C11A00
:1000B000C11AC11AC11AC11AC11AC11AC11AC11A68
:1000C000C11AC11AC11AC11AC11AC11A511A511A38
:1000D000511A511A511A511A511A511A511AC11A58
:1000E000C11AC11AC11AC11AC11AB619501A501A26
:1000F000501A501AC11A5E1A641A6A1A701A761ABD
:100100007C1A821A881A921A9C1AA61AB01AF7191F
:10011000B919C11AC11AC11AC11A451AC11AC11A8C
:10012000C11AC11AC11AC11AC11AC11A4F1A4F1ADB
:100130004F1A4F1AC11A5E1A641A6A1A701A761A7E
:100140007C1A821A881A921A9C1AA61AB01AF719DF
:10015000B919C11AC11AC11AC11A451AF41AF41AE6
:10016000F41AF41AF41AF41AF41AF41AF41AF41A1F
:10017000F41AF41AF41A0B1C0B1C0B1C0B1C0B1C92
:100180000B1C391B431B4D1B571BB51BBF1BCE1B29
:10019000DF1B671D7C1D881D911DA01DC51DCE1D6B
:1001A000171EE01D2B21312137213E214C216E21CC
:1001B0008C21456E746572206D656E752E2E2E0035
:1001C000546F67676C6564206D6963726F50504D42
:1001D00000546F67676C656420696E76657274653C
:1001E000642050504D2100546F67676C6564205443
:1001F00058206D7574696E672100546F67676C6570
:10020000642074656C656D65747279210050726F3D
:10021000746F636F6C206572726F72207769746897
:100220002052580054696D656F7574207768656E4B
:1002300020636F6E6E656374696E6720746F205201
:100240005800507265737320616E79206B65792058
:10025000746F2063616E63656C00436F6E6E6563DF
:1002600074696E6720746F2052582C20706F776508
:100270007220757020746865205258202877697440
:10028000682062696E6420706C7567206966206EF4
:100290006F74207573696E6720616C776179732064
:1002A00062696E642900546F67676C656420276912
:1002B0006D6D656469617465206F75747075742700
:1002C00000546F67676C65642027736C61766520E6
:1002D0006D6F64652700546F67676C6564202761E4
:1002E0006C776179732062696E642700546F676769
:1002F0006C65642050504D206368616E6E656C20A3
:100300006C696D69740053657420525353492069B8
:100310006E6A656374696F6E206368616E6E656C8A
:100320002028303D3D64697361626C652900536526
:10033000742050504D206D696E696D756D20737914
:100340006E630053657420626561636F6E20696E31
:1003500074657276616C0053657420626561636FC9
:100360006E2064656C617900536574206265616319
:100370006F6E206672657175656E637920696E2097
:10038000487A3A20303D64697361626C652C205074
:10039000783D504D52206368616E6E656C20782CFC
:1003A0002046783D465253206368616E6E656C202E
:1003B00078005365742050574D2073746F7020641B
:1003C000656C61792028302064697361626C6564B2
:1003D0002C20312D323535203D3D20302E317320FB
:1003E0002D2035306D696E29005365742050504DB5
:1003F0002073746F702064656C61792028302064EC
:10040000697361626C65642C20312D323535203D75
:100410003D20302E3173202D2035306D696E29003E
:10042000536574206661696C736166652064656CF0
:1004300061792028302064697361626C65642C20C6
:10044000312D323535203D3D20302E3173202D2089
:1004500035306D696E29002A2A2A2A2A2A2A2A2A50
:100460002A2A2A2A2A2A2A2A2A2A2A2A2A2A2A2AEC
:100470002A2A2A2A0052582041636B6564202D20C5
:1004800072657665727420737563636573736675E0
:100490006C21002A2A2A2A2A2A2A2A2A2A2A2A2AAD
:1004A0002A2A2A2A2A2A2A2A2A2A2A2A2A2A2A2AAC
:1004B000002A2A2A2A2A2A2A2A2A2A2A2A2A2A2AC6
:1004C0002A2A2A2A2A2A2A2A2A2A2A2A2A2A00528E
:1004D000582041636B6564202D20757064617465DC
:1004E000207375636365737366756C21002A2A2A0D
:1004F0002A2A2A2A2A2A2A2A2A2A2A2A2A2A2A2A5C
:100500002A2A2A2A2A2A2A2A2A2A0056616C696457
:100510002063686F69636573206172653A205B319F
:100520005D2D5B31365D20286368616E6E656C20E1
:10053000312D31362900536574206F7574707574D0
:1005400020666F7220706F727420005B585D2061AE
:10055000626F7274206368616E67657320616E6498
:10056000206578697420525820636F6E6669670051
:100570005B535D20736176652073657474696E6783
:100580007320746F205258005B525D20726576654F
:1005900072742052582073657474696E6773207486
:1005A0006F2064656661756C747300557365206EA9
:1005B000756D62657273205B312D445D20746F2010
:1005C0006564697420706F727473205B452D515D92
:1005D00020666F722073657474696E677300202DD6
:1005E00020726563656976657220636F6E66696700
:1005F000757261746F722C20727820737720000AF4
:100600000A6F70656E4C52536E67200053657420FC
:1006100073657269616C2062617564726174653AB8
:10062000200056616C69642063686F696365733A82
:100630002031202D20342B34202F2032202D203823
:10064000202F2033202D20382B34202F2034202D14
:10065000203132202F2035202D2031322B34202FF5
:100660002036202D20313600536574204368616E9A
:100670006E656C20636F6E6669673A20005365741F
:100680002044617461726174652028302D32293AEA
:10069000200053657420486F70206368616E6E653A
:1006A0006C7320286D61782032342C207365706162
:1006B000726174656420627920636F6D6D61732966
:1006C0002076616C69642076616C75657320312DCC
:1006D0003235353A2000536574206368616E6E656B
:1006E0006C2073706163696E6720287831306B48C5
:1006F0007A293A200053657420524620706F77653E
:10070000722028302D37293A200053657420524634
:10071000206D6167696320286865782920652E67E8
:100720002E20307844454144463030443A2000532E
:1007300065742062617365206672657175656E63AC
:10074000792028696E20487A293A20005B5A5D207A
:10075000656E746572207265636569766572206383
:100760006F6E66696775726174696F6E2075746902
:100770006C79005B465D20646973706C61792061FF
:10078000637475616C206672657175656E63696509
:10079000732075736564005B525D2063616C6375E3
:1007A0006C6174652072616E646F6D206B65792079
:1007B000616E6420686F70206C697374005B495DC2
:1007C000207265696E697469616C697A6520736508
:1007D0007474696E677320746F20736B65746368DB
:1007E0002064656661756C7473005B585D2072658A
:1007F00076657274206368616E67657320616E64EC
:100800002065786974206D656E75005B535D20739B
:100810006176652073657474696E677320746F20E8
:10082000454550524F4D20616E64206578697420B3
:100830006D656E7500557365206E756D62657273BA
:10084000205B302D395D20746F20656469742070E1
:100850006172616D657465727300202D2053797328
:1008600074656D20636F6E66696775726174696F18
:100870006E000A0A6F70656E4C52536E672000510D
:1008800029204F7574707574206265666F726520DB
:100890006C696E6B20283D465329203A2000502970
:1008A00020536C617665206D6F64652028657870D3
:1008B0006572696D656E74616C293A20004F29205C
:1008C00054696D65642042494E44206174207374FC
:1008D000617274757020203A20004E292050504DCE
:1008E000206F7574707574206C696D69746564200F
:1008F000202020203A200044495341424C454400E6
:100900004D292050504D205253534920746F20637D
:1009100068616E6E656C202020203A20004C2920F2
:1009200050504D206D696E696D756D2073796E63E1
:10093000202875732920203A200044495341424C15
:100940004544004B29204661696C736166652062ED
:100950006561636F6E20696E74762E2028312D32AA
:10096000353573293A20004A29204661696C736144
:10097000666520626561636F6E2064656C617920D5
:1009800028302D323535203D3E20313073202D204A
:100990003135306D696E293A200049292046616958
:1009A0006C7361666520626561636F6E206672714B
:1009B0002E203A200048292050574D2073746F7024
:1009C0002064656C6179202020202020203A2000BE
:1009D00047292050504D2073746F702064656C61FE
:1009E00079202020202020203A200046292046611E
:1009F000696C736166652064656C617920202020D4
:100A00002020203A200050574D206368616E6E65AB
:100A10006C200066756E6374696F6E3A2000292041
:100A2000706F72742000506F776572546F776572C3
:100A300000445446205548462033322D62697420C4
:100A400031306368004F70656E4C52536E67525878
:100A5000206D696E6920342F36636800466C7974A6
:100A6000726F6E2F4F72616E6765525820554846FF
:100A70002038636800525820747970653A20004429
:100A8000697361626C656400487A00203D3D200016
:100A900043616C63756C61746564207061636B6540
:100AA0007420696E74657276616C3A200042292068
:100AB0004D6963726F202868616C66292050504D23
:100AC000202020203A00412920496E766572746505
:100AD000642050504D20696E20202020203A0030A4
:100AE00029204D7574652062757A7A657220286DAB
:100AF0006F73746C79293A003929205365726961E2
:100B00006C2062617564726174653A00736D617224
:100B100074506F7274004672536B79005472616E38
:100B200073706172656E740044697361626C6564B0
:100B30000038292054656C656D657472793A2020FF
:100B40002020202020003729204368616E6E656CCC
:100B500020636F6E6669673A202000362920446161
:100B60007461726174652028302D32293A2020206A
:100B700000352920486F70206368616E6E656C7364
:100B80003A2020202020003429204368616E6E65C1
:100B90006C2073706163696E673A202000332920EE
:100BA000524620706F7765722028302D37293A2001
:100BB0002020003229205246206D616769633A2067
:100BC0002020202020202020003129204261736530
:100BD000206672657175656E63793A202020000089
:100BE00000000700020100000304060000000000EE
:100BF00000000001020408102040800102040810D7
:100C00002001020408102004040404040404040263
:100C10000202020202030303030303000000002395
:100C2000002600290000000000250028002B0000FD
:100C3000000000240027002A0000632E11241FBE9C
:100C4000CFEFD8E0DEBFCDBF13E0A0E0B1E0E4ED30
:100C5000F2E602C005900D92A83CB107D9F716E064
:100C6000A8ECB3E001C01D92A239B107E1F71CE086
:100C7000CCE3DCE004C02297FE010E946C2FCA3353
:100C8000D107C9F70E949F2E0C9468310C94000084
:100C900080917705813019F482E080937705809107
:100CA0007705833019F484E0809377050895A8953B
:100CB0000895DC01ED91FC910190F081E02D099502
:100CC00008952091780530917905382748E0C901C9
:100CD000880F991F37FF06C09C0151E2252750E17C
:100CE000352701C09C01415091F73093790520933D
:100CF0007805089588E380937A0580E092ECA1E07E
:100D0000B0E080937B0590937C05A0937D05B09324
:100D10007E0587E08093870580EC92E9ADEEB9E12E
:100D200080937F0590938005A0938105B093820501
:100D300085E0809388058DEE9EEFADEABEED809351
:100D4000830590938405A0938505B0938605E9E813
:100D5000F5E080E090E0863028F4DC01AE54BC4F32
:100D60002C9101C020E0219301968831910599F7DB
:100D700082E08093A1058AE08093A205089580EC2B
:100D800091EDA8E9BBE18093BF059093C005A093C6
:100D9000C105B093C20580E090E0A0E0B0E580938B
:100DA000C3059093C405A093C505B093C605E7ECB1
:100DB000F5E080E081938F5F8031E1F70895A0E056
:100DC000B0E0E5EEF6E00C94352FD82F0E949A297A
:100DD0006115710581059105C9F30E94D82F109204
:100DE0008305109284051092850510928605C4E053
:100DF000812C912C54018A94C0908305D090840555
:100E0000E0908505F0908605FE2CED2CDC2CCC24A2
:100E10000E94D32FA50194010E94142F6C0D7D1DFB
:100E20008E1D9F1D609383057093840580938505B7
:100E300090938605C15001F7DD2309F450C009E8FD
:100E400015E0E801A12CB12C62E3C62ED12CE12CD7
:100E5000F12C8881882309F442C0B39419F40E94CC
:100E60007A063DC00E94D32FA70196010E94142F3D
:100E7000E1E0E60FA9E8B5E08A2F801B8A1520F48F
:100E80008D918E13F9CFE9CF2091880530E0A0E154
:100E9000B7E20E94AC2E9B01AC01AE2FB0E00E94E5
:100EA000BB2E40907F05509080056090810570902A
:100EB0008205640D751D861D971D4090BF055090DD
:100EC000C0056090C1057090C205461657066806B9
:100ED000790618F2E993A39488E1A812BACFCDB7A6
:100EE000DEB7E0E10C94512F8436910520F4BC016B
:100EF00080E090E017C09C018E3B910528F42A55B4
:100F00003109AAE0B0E00CC0823D910528F4245BD1
:100F10003109A4E6B0E004C02D5C3109A8E5B2E0D7
:100F20000E94AC2EA4E6B0E09B01AC010E94BB2E57
:100F3000089590E08C599F4F0E947407089561E0D6
:100F400086E00E94472A60E086E00E94802A82E0D4
:100F50008093B00085E08093B10061E083E00E945F
:100F6000472A60E083E00E94802A0895CF93DF93B0
:100F7000EC010097E9F061E086E00E94802A9E0182
:100F800040E050E068E478EE81E090E00E94142FA9
:100F90002F3F31054105510529F020F02FEF30E0BA
:100FA00040E050E02093B3008091B000806107C022
:100FB00060E086E00E94802A8091B0008F7E80935E
:100FC000B000DF91CF91089560E08EE00E94472A43
:100FD00061E08FE00E94472A61E080E10E94472A99
:100FE00060E082E00E94472A61E084E00E94472A94
:100FF000089542E050E068E476E080E00E94CA286C
:101000000895E3E0F0E089E080935700E491E67012
:1010100081E0E63009F080E00895CF93DF93C82F98
:101020000E940108882381F0DFB781E08093760574
:10103000F8940E94570688E180936000C093600096
:10104000C1110E945706DFBFDF91CF9108958F92A3
:101050009F92AF92BF92CF92DF92EF92FF92CF9387
:10106000FC01C0A5EC2FE770F0E0E658FC4FA08132
:10107000B0E0C7FF03C024E130E002C02FE030E061
:10108000FC0197A183E1989FF0011124E25CFE4FDF
:1010900080809180A280B380A20FB31F20E43FE143
:1010A0004DE750E00E94C62EA50194010E94F22E49
:1010B0008C2F887149F469017A01E0EDCE0EE7E0EA
:1010C000DE1EE11CF11C1BC0C7FF05C060E47AE80E
:1010D0008CE29EE004C060E07EEE8AEB9BE069015A
:1010E0007A01F8EBCF0EFBE0DF1EE11CF11CA5013D
:1010F00094010E94F22EC20ED31EE41EF51EC701FB
:10110000B60169517C4F8F4F9F4F28EE33E040E08E
:1011100050E00E94F22EA8EEB3E00E94BB2ECF91C9
:10112000FF90EF90DF90CF90BF90AF909F908F9007
:1011300008958F3F910551F048F0811522E0920704
:1011400038F08115934030F482E0089580E00895EE
:1011500081E0089583E00895A0E0B0E0E2EBF8E0DC
:101160000C943E2FEB018A01B82FB695A0E02881A0
:101170003981F80120832A813B8121832C813D81A3
:1011800022832E813F812383688179814A815B811B
:101190002C813D81EE81FF819F2F9295990F990FB0
:1011A000907C272F2370922B252F2370220F220F44
:1011B000922B232F23702295207F922BF80194836A
:1011C0000B5F1F4F2896AF5FBA1788F680FF24C0C9
:1011D000888199810E949908D82E8A819B810E94DA
:1011E0009908E82E8C819D810E949908F82E8E81A5
:1011F0009F810E949908F0E4DF9EA001112490E1F4
:10120000E99E90011124242B282BE4E0FE9EB001DE
:101210001124262BF8012083CDB7DEB7E7E00C942C
:101220005A2F803223E0920708F1883E23E092078C
:1012300040F48F519340E4E096958795EA95E1F765
:101240000895803D27E0920718F48C5D934008953F
:10125000883928E0920768F4885C974074E0969596
:1012600087957A95E1F78D509C4F089580E090E046
:1012700008958FEF93E008958C30910540F4A4E039
:10128000880F991FAA95E1F7885D9C4F0895843FC8
:1012900023E0920718F484529C4F0895811524E0AE
:1012A000920740F48657934FF4E0880F991FFA9500
:1012B000E1F7089580E998E008959C013695279517
:1012C00025753575821B930B9C012373337396959B
:1012D00087959695879583739373820F931F9C01CF
:1012E00054E0369527955A95E1F7280F391F2F704E
:1012F0003F7041E051E0249FC001259F900D349F35
:10130000900D1124892F08954298882319F0000028
:10131000419A02C0000041980000429A00000895DE
:10132000429A000086B14298000081700895CF93E0
:10133000DF93D82F5C9A42985C98C8E08D2F807814
:101340000E948409DD0FC150C9F74298DF91CF9107
:1013500008958F770E9497090895CF93DF93D82F30
:10136000C8E08D2F80780E948409DD0FC150C9F735
:101370004298DF91CF910895CF93DF934298C8E0D0
:1013800080E0D82FDD0F0E9490098D0FC150C9F762
:10139000DF91CF9108950E94A9090E94BC095C9A2F
:1013A0000895A1E0B0E0E7EDF9E00C94432F8068E8
:1013B00069830E9497096981862F0E94AD095C9A12
:1013C0002196E2E00C945F2FCF93C0918305C8274C
:1013D000E82FF0E0E658FA4F678589E70E94D109C7
:1013E0006C2F8DE30E94D1096C2F82E40E94D109F9
:1013F000CF91089586E20E94CB090895CF93DF93A1
:10140000EC016C818CE10E94D1096D818DE10E941B
:10141000D1096E818EE10E94D1096F8180E20E9424
:10142000D109688581E20E94D109698582E20E9422
:10143000D1096A8583E20E94D1096B8584E20E940A
:10144000D1096C8585E20E94D1096D858AE20E94EE
:10145000D1096E858EE60E94D1096F858FE60E94C4
:10146000D109688980E70E94D109698981E70E94D2
:10147000D1096A8982E70E94D109DF91CF9108954D
:10148000CF92DF92EF92FF92CF93DF936B017C01BB
:10149000C11488E3D8068CE9E8068CE1F80628F543
:1014A000C701B60120E836E948E950E00E94F22E73
:1014B000E901689760E879E687E69FEF0E94CE2E03
:1014C0006C0D7D1D8E1D9F1DF2E0660F771F881F1E
:1014D000991FFA95D1F721E732E040E050E00E94F1
:1014E000F22EF22EE32E80E421C0C701B60120E0E7
:1014F0003DE241E351E00E94F22EE901689760E08D
:1015000073ED8EEC9EEF0E94CE2E6C0D7D1D8E1D18
:101510009F1D660F771F881F991F21E732E040E06B
:1015200050E00E94F22EF22EE32E80E66C2F6F71B7
:10153000680F85E70E94D1096E2D86E70E94D109C8
:101540006F2D87E70E94D109DF91CF91FF90EF9037
:10155000DF90CF900895682F8DE60E94D1090895FD
:101560008F929F92AF92BF92CF92DF92EF92FF92B3
:10157000CF93DF93D82F83E00E94CB09809375052A
:1015800084E00E94CB098093740560E086E00E94AD
:10159000D10961E087E00E94D1096FE789E00E94EC
:1015A000D10965E08AE00E94D10962E18BE00E94E6
:1015B000D10965E18CE00E94D1096DEF8DE00E94B8
:1015C000D10960E08EE00E94D109DD2319F08BE2A1
:1015D00091E008C02091A10533E1239FC0011124AF
:1015E000825C9E4F0E94FE096CE880E30E94D10954
:1015F0006FE082E30E94D10962E483E30E94D10993
:101600008091A20587FF02C064E101C06AE084E323
:101610000E94D1096AE285E30E94D1096DE286E366
:101620000E94D10964ED87E30E94D10960E088E35C
:101630000E94D10960E089E30E94D109D11109C05B
:10164000C0908305D0908405E0908505F0908605D4
:1016500007C0C5E9CC2EC1ECDC2EED2CCEEDFC2E66
:10166000CAE38F2C9924AA24BB24682D8C2F0E94B6
:10167000D109682D85E08C0F0E94D109FE2CED2C3C
:10168000DC2CCC24CF5FCE3361F76FEF83E40E9474
:10169000D1096FEF84E40E94D1096FEF85E40E94C5
:1016A000D1096FEF86E40E94D109DD2311F066E0D5
:1016B00002C0609187058DE60E94D10960E089E74C
:1016C0000E94D109609188058AE70E94D10960E0F3
:1016D00083E70E94D10960E084E70E94D109D1111B
:1016E00009C060917F05709180058091810590917E
:1016F000820504C060EC72E98DEE99E10E94400A17
:10170000DF91CF91FF90EF90DF90CF90BF90AF909F
:101710009F908F90089561E087E00E94D10964E274
:101720008EE70E94D10963E088E00E94D10960E061
:1017300088E00E94D10965E087E00E94D10962E05B
:1017400085E00E94D10983E00E94CB098093750552
:1017500084E00E94CB0980937405089583E00E9481
:10176000CB098093750584E00E94CB0980937405B2
:1017700061E087E00E94D1096AE070E080E090E0DB
:101780000E94BD290E948B0B00000895CF92DF922A
:10179000FF920F931F93CF93DF931F92CDB7DEB7C6
:1017A000082F162F8EE399830E94D109F02EC02EA8
:1017B0009981D92E8C2D8F19811738F4F6016191FA
:1017C0006F018FE70E94D109F5CF64E085E00E94A8
:1017D000D10983E00E94CB098093750584E00E94C3
:1017E000CB09809374050E949A29609370057093C9
:1017F0007105809372059093730569E087E00E94FC
:10180000D10981E0809377050F90DF91CF911F91EF
:101810000F91FF90DF90CF9008950F931F930E9438
:10182000C60B80917705813099F40E949A29009126
:101830007005109171052091720530917305601B40
:10184000710B820B930B603A76488140910548F307
:1018500080917705813031F46EE971E086EE95E094
:101860000E94862B1F910F9108950F931F938091D3
:101870007705823021F41092770581E020C08091B5
:1018800077058130D9F40E949A2900917005109152
:1018900071052091720530917305601B710B820BED
:1018A000930B613A76488140910540F061E087E012
:1018B0000E94D1091092770582E001C080E01F915B
:1018C0000F910895CF93DF93EC014AE050E06D2F24
:1018D00070E086EE95E00E94542C6EE286EE95E074
:1018E0000E94582BBE0184E0769567958A95E1F7B2
:1018F0006F7077274AE050E086EE95E00E94542C06
:101900006EE286EE95E00E94582BBE016F7077273D
:101910004AE050E086EE95E00E94542CDF91CF9192
:101920000895D82FC0E0CD1790F4439A299A64E621
:1019300070E080E090E00E94BD294398299864E619
:1019400070E080E090E00E94BD29CF5FECCF6CE2B8
:1019500071E080E090E00E94BD29E4CF0F931F93D7
:10196000CF93DF93EC01062F15E0115051F0CE011B
:101970000E944F31081741F0602FCE010E9457316D
:10198000F4CF82E00E94910CDF91CF911F910F91D3
:101990000895A0E0B0E0EFECFCE00C94352F482E69
:1019A000562EC0E0D0E0612C712CE12CF12C00E02F
:1019B00010E041100CC06090D80586E4689E3001AC
:1019C000112459E1E52EF12C0EEB15E01EC091E03B
:1019D00049120FC06090D805E6E46E9E30011124D4
:1019E000FBE16F0E711C49E2E42EF12C0AE715E0D1
:1019F0000CC082E0481209C028E1622E772473945B
:101A0000EE24E394F12C07ED15E043018C0E9D1EAE
:101A100010927905109278053401A62CA818B12CE3
:101A2000C30101966C01AE14BF04A8F4A00EB11E50
:101A3000511006C0C3010E944F31F501808305C0DB
:101A4000F5016081C3010E94AE0CF50180810E9406
:101A500061063601E2CFC301511018C0C3010E94D4
:101A60004F31B82EC6010E944F312B2D30E0322F5E
:101A70002227282B8091780590917905821793076A
:101A800079F4C0E0D0E05524539493CF36016091AF
:101A900079050E94AE0C60917805C6010E94AE0CDB
:101AA000C05EDE4FC13E92E0D90708F482CF852D9B
:101AB000CDB7DEB7E0E10C94512F61E082E00E94E7
:101AC000C90C089560E082E00E94C90C8091D7059E
:101AD000853020F01092D7050E945D0D8091D705CA
:101AE0008093D805089561E080E00E94C90C61E010
:101AF00081E00E94C90C089560E080E00E94C90C5A
:101B0000882351F060E081E00E94C90C882321F015
:101B100080917A05883349F00E94BF060E947A06B8
:101B200081E00E94DF060E94730D0895882319F05A
:101B30006AEA71E002C06EEA71E086EE95E00E940A
:101B4000862B0895FF920F931F93CF93DF9369EC39
:101B50007BE086EE95E00E94322B40917F0550910C
:101B6000800560918105709182052AE030E086EE63
:101B700095E00E945B2C63EB7BE086EE95E00E9493
:101B8000322B4091830550918405609185057091B9
:101B9000860520E130E086EE95E00E945B2C6DE941
:101BA0007BE086EE95E00E94322B4AE050E06091A7
:101BB000870586EE95E00E94832C67E87BE086EE41
:101BC00095E00E94322B4AE050E06091880586EE55
:101BD00095E00E94832C61E77BE086EE95E00E9411
:101BE000322BC9E8D5E0F12C8E0188818823A9F039
:101BF000FF2031F061EB71E086EE95E00E94552BFD
:101C000021964AE050E0F801608186EE95E00E945E
:101C10004C2CF394F8E1FF12E7CF86EE95E00E949A
:101C2000602B6BE57BE086EE95E00E94322B4AE06C
:101C300050E06091A10586EE95E00E94832C66E459
:101C40007BE086EE95E00E94322BE091A205E770E2
:101C5000F0E0EE0FFF1FEE57FC4F6081718186EEC2
:101C600095E00E94862B61E37BE086EE95E00E9482
:101C7000322B8091A2058871883069F028F4811197
:101C800013C068E27BE00CC0803141F0883161F420
:101C90006CE07BE005C06CE17BE002C066E17BE0CC
:101CA00086EE95E00E94742B68EF7AE086EE95E070
:101CB0000E94322B40917B0550917C0560917D05FF
:101CC00070917E052AE030E086EE95E00E945B2C64
:101CD0006FED7AE086EE95E00E94322B8091C3058D
:101CE00080710E94960D66EC7AE086EE95E00E9487
:101CF000322B8091C30580740E94960D6DEA7AE0C4
:101D000086EE95E00E94322B8091C30580720E947E
:101D1000960D60E97AE086EE95E00E94322B8AE724
:101D200095E00E942708AB01BC012AE030E086EE76
:101D300095E00E943D2C6BE87AE086EE95E00E94EB
:101D4000322B8AE795E00E9427089B01AC0160E4F2
:101D500072E48FE090E00E94F22EBA01A9012AE01D
:101D600030E086EE95E00E943D2C68E87AE086EE51
:101D700095E00E94742BCDB7DEB7E5E00C945C2FA4
:101D80008F929F92AF92BF92CF92DF92EF92FF928B
:101D9000811107C06FE77AE086EE95E00E94742B10
:101DA0002FC090E00E94740724E630E040E050E04D
:101DB0000E94F22ECA01B9012AE030E040E050E072
:101DC0000E94F22E49015A016B017C012AE030E0A9
:101DD000B501A40186EE95E00E943D2C6EE286EEF0
:101DE00095E00E94582B2AE030E0B701A60186EE6C
:101DF00095E00E943D2C63E786EE95E00E94982BCB
:101E0000FF90EF90DF90CF90BF90AF909F908F901A
:101E100008951F93CF93DF9365E77AE086EE95E010
:101E20000E94322B8091A305813041F46CE57AE069
:101E300086EE95E00E94742B10E050C0823019F4B9
:101E400065E47AE0F5CF843019F461E37AE0F0CF0D
:101E5000853091F766E27AE0EBCFC12FD0E0C93050
:101E6000D1050CF441C068E3610F86EE95E00E9455
:101E7000582B6EE17AE086EE95E00E94322BBE018F
:101E80006F5F7F4F4AE050E086EE95E00E941C2C89
:101E900063E17AE086EE95E00E94322BCD55DA4F71
:101EA000E981E03218F566E07AE086EE95E00E947E
:101EB000322B8981803130F06DE673E086EE95E05B
:101EC0000E94552B69816F7070E06F5F7F4F4AE011
:101ED00050E086EE95E00E94252C1F5F80914C0516
:101EE000181708F4BACF0FC061E3BECFEF70F0E06F
:101EF000EE0FFF1FEE56FC4F6081718186EE95E07C
:101F00000E94862BEACF6BEE79E086EE95E00E9488
:101F1000322B8091BB050E94C00E60ED79E086EE09
:101F200095E00E94322B8091BC050E94C00E65EBAB
:101F300079E086EE95E00E94322B8091BD050E94EB
:101F4000C00E6AE979E086EE95E00E94322B40915E
:101F5000B3055091B4056091B5057091B605411572
:101F600051056105710539F12AE030E086EE95E012
:101F70000E945B2C67E679E086EE95E00E94322BAA
:101F80008091B7050E949907AB01BC012AE030E0BF
:101F900086EE95E00E945B2C63E479E086EE95E0A6
:101FA0000E94322B4AE050E06091B80586EE95E041
:101FB0000E94832C06C06AE379E086EE95E00E94D9
:101FC000742B6DE179E086EE95E00E94322B6091F2
:101FD000B9057091BA054AE050E086EE95E00E949E
:101FE0006D2C60E079E086EE95E00E94322B6091E6
:101FF000B205603450F470E06F5F7F4F4AE050E00C
:1020000086EE95E00E94252C06C067EF78E086EE0C
:1020100095E00E94742B6AED78E086EE95E00E94D0
:10202000322B8091B10580FF03C063EB71E002C0E9
:1020300067EB71E086EE95E00E94862B6DEB78E011
:1020400086EE95E00E94322B8091B10582700E944D
:10205000960D6EE978E086EE95E00E94322B809135
:10206000B10584700E94960D6FE778E086EE95E0EA
:102070000E94322B8091B10588700E94960DDF91ED
:10208000CF911F9108950F931F93CF93DF932091CA
:1020900049052F3FA9F56FEF75E086EE95E00E94A8
:1020A000322B88E893E00E94620C6EED75E086EEBC
:1020B00095E00E94322B80914A0590914B050E9439
:1020C000620C6BEA75E086EE95E00E94742B68E87E
:1020D00075E086EE95E00E94742B60E775E086EE71
:1020E00095E00E94742B6BE475E086EE95E00E940B
:1020F000742B86EE95E00E94602B0E94090F68C049
:1021000012160CF065C0332727FD309580914C05E1
:1021100090E0821793070CF45BC066E375E086EEEF
:1021200095E00E94322B60914905772767FD7095F5
:102130004AE050E086EE95E00E94252C6BE075E0C9
:1021400086EE95E00E94322B10E008E280914D056A
:102150001817D0F5C12FD0E0CC0FDD1FC25BDA4FCE
:10216000288130E080914905992787FD9095019756
:102170002817390739F56BEB71E086EE95E00E9480
:10218000552B4AE050E0602F86EE95E00E944C2CE3
:102190006FEB71E086EE95E00E94552BE981EF70C0
:1021A000F0E0EE0FFF1FEE56FC4F6081718186EE6E
:1021B00095E00E94552B63EC71E086EE95E00E945D
:1021C000552B0F5F1F5FC2CF86EE95E00E94602BFC
:1021D000DF91CF911F910F910895FF920F931F935D
:1021E000CF93DF93C9E8D5E0F12C8E018881882355
:1021F000D1F165EC71E086EE95E00E94552B4AE046
:1022000050E06F2D86EE95E00E944C2C62ED71E05F
:1022100086EE95E00E94552B2196F801208130E052
:10222000A0E1B7E20E94AC2E9B01AC01A091880511
:10223000B0E00E94BB2EAB01BC0180917F05909164
:102240008005A0918105B0918205480F591F6A1F32
:102250007B1F2AE030E086EE95E00E945B2CF39431
:10226000F8E1FF12C2CFCDB7DEB7E5E00C945C2FEA
:102270001092E30485E6E4EEF4E0DF011D928A9516
:10228000E9F70895CF93C82F8F3719F0883009F0F8
:1022900045C0E091E304EE23D9F1E150E093E3047B
:1022A000F0E0EC51FB4F10826DE070E086EE95E0BF
:1022B0000E945906C0E08091E304C81760F4EC2F37
:1022C000F0E0EC51FB4F608170E086EE95E00E94FB
:1022D0005906CF5FF0CF60E270E086EE95E00E9495
:1022E00059066DE070E086EE95E00E945906C0E068
:1022F0008091E304C81778F5EC2FF0E0EC51FB4F28
:10230000608170E086EE95E00E945906CF5FF0CFC5
:1023100067E086EE95E00E94582B1DC08B3119F4C2
:102320000E9438111AC08D30C1F08A30B1F080910E
:10233000E304843668F76C2F70E086EE95E00E9427
:102340005906E091E30481E08E0F8093E304F0E00E
:10235000EC51FB4FC08380E001C081E0CF91089534
:10236000CF93C82F0E949A296093CC047093CD0418
:102370008093CE049093CF04C093E104CC2329F042
:1023800040E051EE60E070E004C040E855E260E0FB
:1023900070E086EE95E00E94E22DCF910895909135
:1023A000D004492F4F7050E0BA016F5F7F4F292F43
:1023B00030E0E4E035952795EA95E1F76217730779
:1023C00059F0FA01EF52FB4F808381E0890F8F7043
:1023D000907F892B8093D00408956EE770E086EE9D
:1023E00095E00E9459060895A3E1B1E0EAEFF1E11A
:1023F0000C94362FE9E8F5E0712C8191882321F0C7
:10240000739428E17212F9CF66ED71E086EE95E0E3
:102410000E94862B4AE050E0672D86EE95E00E94F0
:10242000832C80E00E94B00A0E948B0B8E010E5F0D
:102430001F4FC12CD12C7601C39466246A945C2C66
:102440000E948E294B015C012091880530E0A0E1BB
:10245000B7E20E94AC2E9B01AC01C701B6010E94FD
:10246000CE2E20917F0530918005409181055091BD
:102470008205620F731F841F951F2091BF05309145
:10248000C0054091C1055091C2052617370748077E
:10249000590718F4F80160822AC08C2D0E94E409C3
:1024A00061E070E080E090E00E94BD29F8011082B8
:1024B0000E948E29681979098A099B09643F714035
:1024C0008105910540F40E94FA09F801908198175E
:1024D00078F78083EDCF85B150FE05C08B7D85B93F
:1024E000439A299A04C0846285B9439829982FEFAA
:1024F000C21AD20AE20AF20A0F5F1F4F8FEFC81604
:10250000D104E104F10409F09ACFCE019395FC01C6
:10251000D82E7FEF68EC2E2F281B271510F051E0E6
:1025200056C0DE01129651E02FEF41E03D91321787
:1025300010F0322F01C0452F5F5F5F3F11F0232F56
:10254000F5CF4193242F30E0A1E0B0E0AC0FBD1FE8
:10255000A20FB31F5C93413079F0DE01A20FB31FCD
:102560005C93423049F0AFEFBFEFAC0FBD1FA20F3D
:10257000B31F6C934E3F78F6A2E0B0E0AC0FBD1FE6
:10258000A20FB31F7C934D3F30F6A3E0B0E0AC0F39
:10259000BD1FA20FB31F6C93BECF452F242F30E079
:1025A000FC01E20FF31F6081AFEFB0E0AC0FBD1F85
:1025B000A20FB31F2C91621748F44150DC01A40F05
:1025C000B11D2C9120836C934111E8CF5F5F5715AB
:1025D00020F3372D369520E0231770F4DC01A20F8D
:1025E000B11D4C91522F530FFC01E50FF11D50818D
:1025F0005C9340832E5FF0CFF9E8EF2EF5E0FF2EDD
:102600008C01802F8D19871598F4F801C1908F01E6
:102610004AE050E06C2D86EE95E00E944C2C6CE276
:1026200086EE95E00E94582BF701C1927F01E9CF19
:1026300086EE95E00E94602B81E0CD5EDE4FEFE0FC
:102640000C94522F1F920F920FB60F9211241F93CA
:102650002F933F934F935F936F937F938F939F93AA
:10266000AF93BF93CF93DF93EF93FF93C091860017
:10267000D091870080918704909188042091A904CB
:10268000211155C09E01281B390B8091C3059091E3
:10269000C405A091C505B091C60585FD02C036955B
:1026A0002795253C49E03407B8F140910A0150E0F4
:1026B00060E070E02CE1B695A795979587952A95EF
:1026C000D1F70097A105B10521F481E090E0A0E0E9
:1026D000B0E084179507A607B707D8F480910A01E0
:1026E0008F3FB9F040E080910A01481780F4842FB1
:1026F00090E0880F991FFC01E757FB4F2081318143
:10270000FC01E55FFE4F318320834F5FECCF1092D9
:10271000AA0410920A010BC02D3B82E0380720F07A
:1027200080910A018031D8F08FEF80930A01D09315
:102730008804C0938704FF91EF91DF91CF91BF91FF
:10274000AF919F918F917F916F915F914F913F9149
:102750002F911F910F900FBE0F901F901895109101
:102760000A0181E0810F80930A01C9010E941109C9
:10277000E12FF0E0EE0FFF1FE757FB4F91838083BF
:10278000D6CF83E0809380008AE980938100809196
:10279000C30586FD05C0809181008064809381001F
:1027A0008FEF9FEF909389008093880080916F0056
:1027B000806280936F000895CF93DF930E94620D33
:1027C0008091D805843039F58BE00E94B32AC1E0AE
:1027D000D0E0892B11F4C0E0D0E08CE00E94B32A55
:1027E000892B19F082E090E002C080E090E08C2B11
:1027F0009D2B8230910539F08330910539F0019796
:1028000039F481E006C01092D80505C082E001C00D
:1028100083E08093D805DF91CF9108956F3018F051
:1028200086958058089589E0689F802D1124089529
:10283000A0E0B0E0EEE1F4E10C943D2FC82F0E943F
:102840009A29009138041091390420913A0430916A
:102850003B046B017C01C01AD10AE20AF30A97011A
:10286000860149E8C41643E1D406E104F10410F0FE
:1028700010923C04609338047093390480933A04B6
:1028800090933B042091A9048FEF820F8230E8F5EA
:10289000E0913C04EE2309F46EC1E13011F482E0D2
:1028A000D8C1E03178F581E08E0F80933C04F0E0F0
:1028B000E757FB4FC083803109F0D4C1EBE8F4E067
:1028C000213029F4A181A695A695808108C0808138
:1028D0009181A92FA695A695A69596958795A03145
:1028E00048F4B0E090E0AA0FBB1FA55FBE4F119661
:1028F0009C938E931092AA04329684E0E939F807EB
:10290000F9F6B0C110923C04ADC1233009F023C1E7
:10291000E0913C04E11118C0CF3009F011C10E94D0
:102920008E290091B7041091B8042091B904309118
:10293000BA04601B710B820B930B62307105810529
:10294000910508F089C1FCC0E73148F481E08E0FA1
:1029500080933C04F0E0E857FB4FC083F1C0E731BF
:1029600009F0ECC0C111EAC040E050E0ABE0CA01A0
:10297000B3E0880F991FBA95E1F7A49F9001A59F36
:10298000300D1124F901E757FB4F6081E1817E2F63
:10299000777075956795FC01EE0FFF1FE55FFE4FA1
:1029A00071836083F901E657FB4FB081B695B69508
:1029B000B695E181FE2FF295FF0FF07E6F2F6B2B06
:1029C000E695E695E6957E2F777075956795FC01FF
:1029D000EE0FFF1FE35FFE4F71836083F901E55740
:1029E000FB4FB081B295B695B695B370C181DC2F1F
:1029F000DD0FDD0F6D2F6B2BC295C695C695C3708D
:102A0000E281E170EE0FEE0F7E2F7C2B75956795BE
:102A1000FC01EE0FFF1FE15FFE4F71836083F90140
:102A2000E357FB4FB081B695E181FE2FF795FF2765
:102A3000F7956F2F6B2BE6957E2F777075956795C1
:102A4000FC01EE0FFF1FEF5EFE4F71836083F90103
:102A5000E257FB4FB081B295BF70E181FE2FF29536
:102A6000F07F6F2F6B2BE295EF707E2F777075954F
:102A70006795FC01EE0FFF1FED5EFE4F71836083D3
:102A8000F901E157FB4FB081BB1FBB27BB1FC181C1
:102A9000DC2FDD0F6D2F6B2BCC1FCC27CC1FE281E1
:102AA000E370EE0F7E2F7C2B75956795FC01EE0F82
:102AB000FF1FEB5EFE4F71836083F901EF56FB4F02
:102AC000B081B695B695E181FE2FF295FF0FFF0F0D
:102AD000F07C6F2F6B2BE695E6957E2F77707595C2
:102AE0006795FC01EE0FFF1FE95EFE4F7183608367
:102AF000F901EE56FB4F20812295269527703181F2
:102B0000E32FEE0FEE0FEE0F6E2F622B732F7295E9
:102B10007695777075956795FC01EE0FFF1FE75E60
:102B2000FE4F718360834F5F5F4F4230510509F064
:102B30001ECF80919F0483FF1092AA0410923C0440
:102B40000E948E296093B7047093B8048093B904EF
:102B50009093BA0487C0243009F084C060913C048B
:102B600061110BC0C83AB1F4109279051092780542
:102B700088EA0E94610681E06CC0613019F4C0935C
:102B8000370404C0623031F4C09336048C2F0E94A5
:102B900061065AC0E09136042E2F30E0220F331F19
:102BA000462F50E0C9010296841795073CF0633226
:102BB00068F7FA01EA57FB4FC083E8CF2D5F3F4F1C
:102BC0008C2F90E06091780570917905421753073A
:102BD00049F4982F88278627972790937905809323
:102BE000780532C06817790769F58091370481301C
:102BF00049F5E13118F080E180933604F090360415
:102C0000CAE8D4E000E010E00F15D0F4FE013197DF
:102C1000808190E0982F88272881822B63E0969509
:102C200087956A95E1F70E941109F801EE0FFF1FE1
:102C3000E55FFE4F918380830F5F1F4F2296E4CFA5
:102C40001092AA0410923C0480913C04882351F015
:102C50008F5F80933C0406C080913C048F5F80931B
:102C60003C046ECFCDB7DEB7E8E00C94592FCF937C
:102C7000DF93E82FF0E0E254FA4FE185E03150F4C1
:102C8000F894F0E0EE0FFF1FE55FFE4F8081918129
:102C900078945DC08EE08E0F8B3058F4F0E0E25FE8
:102CA000F10924E62E9FC0012F9F900D11240C9650
:102CB0004EC0E03F09F446C038F4E13181F0E23122
:102CC00091F0E03139F409C0ED3FB1F1EE3FB9F1D7
:102CD000E13F79F180E092E03AC082E101C083E116
:102CE0000E94DC2A34C08BE00E94B32AC1E0D0E00D
:102CF000892B11F4C0E0D0E08CE00E94B32A892B2C
:102D000019F082E090E002C080E090E08C2B9D2BD7
:102D10008230910541F08330910541F00197A9F08F
:102D200086EA92E014C08CE090E011C089E591E061
:102D30000EC086E090E00BC08AEF93E008C08FEFF2
:102D400093E005C080E090E002C084EF93E0DF9163
:102D5000CF910895A2E2B0E0E0EBF6E10C94332FBE
:102D60009E012F5F3F4F80E1D9011D928A95E9F7BF
:102D700064E072E086EE95E029A33AA30E94862BD8
:102D80000E94AE0B1D8A1E8A1F8A188E312C212CA0
:102D900000E0812C912C540170E4472E71EE572EE7
:102DA0007DE9672E78E1772EE0E5CE2EE3ECDE2E8E
:102DB000E12CF12C84EF91E0A0E0B0E08D8F9E8FAC
:102DC000AF8FB8A380EC91EDA8E9BBE1898F9A8F12
:102DD000AB8FBC8F80E491EEADE9B8E1898B9A8B23
:102DE000AB8BBC8B86EE95E00E949A2C892B09F464
:102DF000E1C086EE95E00E94C72C9C0133272C325F
:102E0000310509F442C0ACF42332310509F0ABC0FE
:102E100019821A821B821C821D821E821F821886C2
:102E200019861A861B861C861D861E861F86188A92
:102E300060C02434310529F02335310509F4B2C0CE
:102E400092C064E486EE95E00E94582B2AE030E0C0
:102E500040E451EE6DE978E186EE95E00E94E62BC4
:102E60006CE286EE95E00E94582B2AE030E040ECC0
:102E700051ED68E97BE186EE95E00E94E62B6CE27D
:102E800086EE95E00E94982BADCF0F5F043009F0DD
:102E9000A9CF29813A814B815C81A8EEB3E00E94E1
:102EA000BB2E698B7A8B8B8B9C8B2D813E814F81C6
:102EB00058850E94BB2E698F7A8F8B8F9C8F2985B6
:102EC0003A854B855C852D8F3E8F4F8F58A32D857E
:102ED0003E854F8558890E94BB2E6B017C01603274
:102EE0003EE473078105910530F462E38CE10E94B2
:102EF000D10900E077CF603345E77407810591057C
:102F000010F462E2F3CF60345CE975078105910546
:102F100010F466E2EBCF80E5C81683ECD806E10436
:102F2000F10410F462E1E2CF90E6C9169AEED906F8
:102F3000E104F10410F465E1D9CFA0E7CA16A1E1DC
:102F4000DA06A1E0EA06F10410F461E0CFCFB0EABE
:102F5000CB16B6E8DB06B1E0EB06F10410F463E053
:102F6000C5CF65E0C3CF10ED180F1A3008F03ACF87
:102F7000E1E0F0E0EC0FFD1F24E0029FE00DF11D09
:102F800011242081318142815381AAE0B0E00E9466
:102F9000BB2E610F711D811D911D60837183828322
:102FA000938320CF49885A886B887C88812C912C08
:102FB000540118CF81149104A104B10489F4C30110
:102FC000B2010E94400A61E070E080E090E00E945F
:102FD000BD291D8A1E8A1F8A188E312C22242A940C
:102FE0008D8D9E8DAF8DB8A188169906AA06BB0659
:102FF000D0F40E94FA092D893E894F89588D280FF7
:10300000311D411D511D2D8B3E8B4F8B588F381616
:1030100008F4382E821508F4282E3FEF831A930AFD
:10302000A30AB30A56C0C301B20128EE33E040E060
:1030300050E00E94F22EBA01A9012AE030E086EEAB
:1030400095E00E943D2C6CE286EE95E00E94582BA4
:103050004AE050E0632D86EE95E00E944C2C6CE235
:1030600086EE95E00E94582B6D897E898F89988D18
:10307000A50194010E94F22EBA01A9012AE030E0D4
:1030800086EE95E00E943D2C6CE286EE95E00E9473
:10309000582B4AE050E0622D86EE95E00E944C2CC1
:1030A0006CE286EE95E00E94982B4C0C5D1C6E1C29
:1030B0007F1C898D9A8DAB8DBC8D84159505A605D9
:1030C000B70520F449885A886B887C88812C912C1C
:1030D000540129893A894B895C89283E334041054E
:1030E000510509F07FCEA296E2E10C944F2FACE19E
:1030F000B0E0EDE7F8E10C943D2F0E949A296B01B6
:103100007C0181E00E94B00A14E703E0198361E0CA
:10311000CE0101960E940D0C009377050E948B0B47
:103120006AEF70E080E090E00E94BD298091770511
:10313000833089F486EE95E00E949A2C892B59F40D
:103140000E949A296C197D098E099F096038734C79
:10315000894C9140D8F280917705833009F44FC0B3
:103160008FE70E94A9090E94BC098983843511F068
:1031700083E05CC00E94BC0910924A0580934B0515
:103180000E94BC0920914A0530914B05280F311D42
:1031900030934B0520934A050E94BC0980934C054F
:1031A0000E94BC0980934D05813110F7F12C0F2D41
:1031B00010E080914D0590E0880F991F08171907BE
:1031C00040F40E94BC09F801E25BFA4F8083F3945B
:1031D000EECF80E7898361E0CE0101960E940D0C5D
:1031E00083E0809377050E948B0B62E370E080E0C0
:1031F00090E00E94BD2980917705833011F482E030
:1032000015C08FE70E94A9090E94BC0989838035F7
:1032100009F0AECF03EA15E00E94BC09F8018193E2
:103220008F01F5E00E3B1F07B9F781E06C96E8E0EF
:103230000C94592F80914905992787FD9095A92FC6
:10324000B92FFC013196EB30F10508F066C0EC5C5B
:10325000FF4F0C946A2F62E778E086EE95E00E94BB
:10326000742B88E893E00E94620C6AE578E086EEB1
:1032700095E00E94742B65E378E086EE95E00E946D
:10328000742B6BE078E086EE95E00E94742B6AEE7A
:1032900077E086EE95E00E94742B6DEB77E086EE8A
:1032A00095E00E94742B67E977E086EE95E00E9436
:1032B000742B63E777E086EE95E00E94742B6CE454
:1032C00077E086EE95E00E94742B86EE95E00E94F2
:1032D000602B0E94A20D21C06FE277E01AC06AE065
:1032E00077E017C065EF76E014C066ED76E011C0B8
:1032F00062E976E00EC06DE776E00BC068E676E046
:1033000086EE95E00E94742B62E276E002C06CE0EB
:1033100076E086EE95E00E94742B6AE070E080E033
:1033200090E00E94BD2986EE95E00E949A2C892BA0
:1033300029F086EE95E00E94C72CF5CF0895ACE108
:10334000B0E0E5EAF9E10C943D2F909149059F3FEB
:1033500009F023C1482F50E0FA013A97EF36F10502
:1033600008F00FC1E15CFF4F0C946A2F61E172E03D
:10337000A0C06DE172E086EE95E00E94862B85E7A5
:1033800089838BE1E3EAF5E0DE01129601900D926C
:103390008A95E1F76CE1CE0101960E940D0C0E9426
:1033A0008B0B83E08093770568EC70E080E090E021
:1033B0000E94BD2980917705843009F0E2C08FE733
:1033C0000E94A9090E94BC098983853509F0D9C0EA
:1033D0006DEE74E086EE95E00E94742B6FEC74E065
:1033E00086EE95E00E94742B61EB74E096C065E375
:1033F00072E086EE95E00E94862B89E6898361E083
:10340000CE0101960E940D0C0E948B0B83E08093ED
:10341000770568EC70E080E090E00E94BD29809123
:103420007705843009F0ADC08FE70E94A9090E949A
:10343000BC0989838E010E5F1F4F7E014DE1E40EB2
:10344000F11C0E94BC09F80181938F01EE15FF0564
:10345000C1F78BE1FE013296A3EAB5E001900D922F
:103460008A95E1F78981893409F08BC063E974E0BA
:1034700086EE95E00E94742B65E774E086EE95E099
:103480000E94742B67E574E048C06FE472E086EE3A
:1034900095E00E94862B8EEF8093490572C0805282
:1034A0008750805390914C05981708F066C06EE5E0
:1034B00072E086EE95E00E94862B63C084E18093E3
:1034C000490560E274E029C085E18093490569EE11
:1034D00073E023C086E18093490562EB73E01DC071
:1034E00087E18093490568E673E017C088E180931F
:1034F000490567E573E011C089E18093490563E4FC
:1035000073E00BC08AE1809349056EE273E005C069
:103510008BE18093490566E073E086EE95E00E94BA
:10352000742B2FC06CEE72E086EE95E00E94742B37
:103530008091B10591E01DC066ED72E086EE95E0E8
:103540000E94742B8091B10592E013C061EC72E08F
:1035500086EE95E00E94742B8091B10594E009C03D
:1035600066EA72E086EE95E00E94742B8091B105C8
:1035700098E089278093B1058FEF809349050E94D9
:10358000431086EE95E00E949A2C892B09F45BC1CA
:1035900086EE95E00E94C72CF4CF0E94421188234A
:1035A00009F451C18091E304811104C08FEF80932D
:1035B000490541C140E050E060E070E084EE94E0F5
:1035C0000E94E12F40914905042F112707FD109516
:1035D000212F312FF8013197EB31F10508F01BC194
:1035E000E255FF4F0C946A2F552747FD50952091C7
:1035F0004C0530E0241735070CF40DC18B019C01FC
:103600000150110921093109003211052105310547
:1036100058F0C0904D05EFE4F5E0F12CD12CA8E274
:10362000EA2E415051090FC0FA01ED55FA4F615091
:103630006083D9C0DF0111972C9130E02417350742
:1036400029F0F3943296FC10F5CFCBC00E2D10E08C
:1036500020E030E0061717072807390741F42081DA
:10366000DA01AD55BA4F11962C93DD24D394E3942F
:10367000E8CF6F3F71058105910511F008F0CBC0CF
:103680006093BB05B0C06F3F71058105910511F0D6
:1036900008F0C1C06093BC05A6C06F3F71058105ED
:1036A000910511F008F0B7C06093BD059CC0209152
:1036B000E40420622037E9F440E050E060E070E08C
:1036C00085EE94E00E94E12F9B01AC01DC01CB016F
:1036D0000197A109B1090897A105B10508F0AEC08D
:1036E000A4EDB0E30E94BB2E6A5E7C4A8A46954EEA
:1036F00024C02636E9F440E050E060E070E085EE5A
:1037000094E00E94E12F9B01AC01DC01CB01019709
:10371000A109B1090797A105B10508F08FC0A8EA72
:10372000B1E60E94BB2E645E7C438E46944E05C07B
:10373000611571058105910579F08B019C0100549B
:10374000114E2D4938410138F0EF1F07FAEF2F07CE
:10375000F2E03F0708F05FC06093B3057093B405D3
:103760008093B5059093B6053EC06F3F7105810506
:10377000910511F008F04FC06093B70534C08B017C
:103780009C0101501109210931090F3F1105210543
:10379000310508F040C06093B80525C08B019C013D
:1037A000045C1940210931090D344DE1140721054C
:1037B000310528F47093BA056093B90514C06115FA
:1037C00071058105910521F48FEF8093B2050BC03F
:1037D0006134710581059105F0F461506093B20583
:1037E00002C0DD20C1F08091E20481111AC08091F5
:1037F000830590918405A0918505B0918605019679
:10380000A11DB11D8093830590938405A093850528
:10381000B093860506C060E772E086EE95E00E94F0
:10382000862B0E9438118FEF809349056AE086EE5F
:1038300095E00E94982B0E94431005C061E070E063
:1038400080E090E07ACF6C96E8E00C94592F6AE51E
:1038500072E086EE95E00E94742B62E472E086EEE0
:1038600095E00E94742B86EE95E00E949A2C892B9D
:1038700031F086EE95E00E94C72C0E949F190E94AD
:103880007718823029F0833051F46DE072E002C085
:1038900064E272E086EE95E00E94742B08958FEF4B
:1038A000809349051092E2040E94431080914905DB
:1038B0008E3F69F086EE95E00E949A2C892BB1F339
:1038C00086EE95E00E94C72C0E949F19EFCF0895C5
:1038D0000F931F93109149051F3F09F0D2C08934FF
:1038E00009F457C000F5883309F469C058F48033EF
:1038F00009F477C008F061C08B3109F440C081320F
:10390000B1F1B9C0813409F487C030F4893309F4C6
:1039100066C0803461F1AFC0823409F48EC0863451
:1039200009F448C0A8C0823609F487C078F4883505
:1039300031F128F48235C1F18335E1F09CC08A353C
:1039400009F494C0813609F467C095C0823761F1EB
:1039500028F4863679F18936E1F08DC0883779F020
:103960008A3709F483C0833709F085C003C061E159
:1039700072E015C00E94730D6EE872E004C00E94F0
:103980007C0D68EA72E086EE95E00E94862B8EEF51
:1039900070C00E947A060E94BF0667EC72E086EE55
:1039A00095E00E94862B67C081E00E94DF0660EEF2
:1039B00072E0F5CF0E94ED105EC080535AC06AEFEE
:1039C00071E086EE95E00E94742B9091A20588E04C
:1039D000890F8871977E892B8093A2051AC089E090
:1039E00048C067EE71E086EE95E00E94742B8091EE
:1039F000C3059091C405A091C505B091C60520E10D
:103A000082278093C3059093C405A093C505B09306
:103A1000C605109349052FC061ED71E086EE95E073
:103A20000E94742B8091C3059091C405A091C50597
:103A3000B091C60540E4842710C060EC71E086EECA
:103A400095E00E94742B8091C3059091C405A091CC
:103A5000C505B091C60520E282278093C3059093E7
:103A6000C405A093C505B093C60502C00E94271CDB
:103A70008FEF80934905809149058E3F09F0D4C0AE
:103A8000DDC00E944211882309F4D8C08091E3046C
:103A9000811104C08FEF80934905C6C040E050E01B
:103AA00060E070E084EE94E00E94E12F009149050F
:103AB000112707FD1095212F312FF8013197E9309B
:103AC000F10508F0B4C0E753FF4F0C946A2F8B0147
:103AD0009C010154114E2D4938410F37104F2A4F88
:103AE000324008F0A4C060937F05709380058093F6
:103AF00081059093820577C0609383057093840558
:103B0000809385059093860581E08093E2046BC0E5
:103B1000683071058105910508F089C060938705BB
:103B200062C08B019C0101501109210931090A3041
:103B300011052105310508F07AC06093880553C04E
:103B400061EB71E084EE94E00E941B3110E000977D
:103B500099F00E94F530009779F0183130F4E12F98
:103B6000F0E0E658FA4F87871F5F61EB71E080E075
:103B700090E00E941B31EBCF1831A8F5E12FF0E067
:103B8000E658FA4F17861F5FF7CF6530710581053C
:103B9000910508F04CC06093A10525C08B019C01E4
:103BA000015011092109310906301105210531059E
:103BB000F0F52091A205287F262B2093A20513C0A3
:103BC0008B019C0101501109210931090115124C89
:103BD0002140310560F560937B0570937C058093EF
:103BE0007D0590937E058091E204811113C0809140
:103BF000830590918405A0918505B0918605019675
:103C0000A11DB11D8093830590938405A093850524
:103C1000B09386050E9438118FEF809349056AE0C2
:103C200086EE95E00E94982B0E941A1907C060E763
:103C300072E086EE95E00E94862BECCF1F910F91EB
:103C400008958FEF809349051092E2040E941A199B
:103C5000809149058E3F69F086EE95E00E949A2C8E
:103C6000892BB1F386EE95E00E94C72C0E94681C58
:103C7000EFCF6AE070E080E090E00E94BD2986EE20
:103C800095E00E949A2C892B29F086EE95E00E94FF
:103C9000C72CF5CF0895CF93C82F682F86EE95E0F7
:103CA0000E94F42C90916E059C2790936E05CF9105
:103CB0000895A1E0B0E0EFE5FEE10C94432F998375
:103CC0000E944B1E9981892F0E944B1E2196E2E093
:103CD0000C945F2F1F93CF93DF93182FEB0110925B
:103CE0006E0565EB70E086EE95E00E94590662E68F
:103CF00070E086EE95E00E945906812F0E944B1ECF
:103D0000CE010E94591EDF91CF911F9108956091BD
:103D10006E0586EE95E00E94F42C0895A1E2B0E0D5
:103D2000E4E9FEE10C943F2F7B018A018C3009F419
:103D300052C108F040C0863009F4BCC018F5833089
:103D400009F491C070F4813009F472C0823009F036
:103D500049C26BE170E082E00E946A1E03EA15E04E
:103D600078C0843009F487C0853009F03BC2609187
:103D70004D0570E0660F771F85E00E946A1E0EE415
:103D800015E086C0893009F4A7C070F4873009F4C3
:103D90009BC0883009F026C261E070E088E00E9494
:103DA0006A1E8091D80524C28A3009F4CAC08B30BB
:103DB00009F4F1C017C28A3609F474C1D8F4873601
:103DC00009F439C138F4853609F40DC1863609F491
:103DD0001EC108C2883609F436C1893609F002C20C
:103DE00061E070E089E60E946A1E0E947A060E94E5
:103DF000BF06F6C18D3609F4D3C138F48B3609F409
:103E000090C18C3609F499C1EDC18E3609F4DDC13B
:103E1000873C09F0E7C161E070E087EC0E946A1E10
:103E200081E00E944B1E0E94871E10926F05E4C124
:103E300069E270E081E00E946A1E0AE715E0F8017D
:103E400081918F010E944B1EF5E0033A1F07B9F7DD
:103E5000D1C1F80181918F010E944B1EF5E00E3B0C
:103E60001F07B9F7C7C161E070E083E00E946A1ED6
:103E70000E947718BDC161E070E084E00E946A1E74
:103E800081E00E944B1E0E94871E0E94AA16B4C1A8
:103E900080914D0590E0880F991F98012E54354070
:103EA0002817390708F0A6C1F80181918F010E94F7
:103EB0004B1EEECF62E070E086E00E946A1E88E84A
:103EC00093E00E94591E96C161E070E087E00E9475
:103ED0006A1E80914C058CC186E6898361E0CE0123
:103EE00001960E940D0C0E948B0B83E08093770556
:103EF00068EC70E080E090E00E94BD298091770539
:103F00008430D9F48FE70E94A9090E94BC098983F3
:103F1000863469F460E270E089E00E946A1E10E273
:103F20000E94BC090E944B1E1150D1F763C161E091
:103F300070E089E00E946A1E53C161E070E089E090
:103F400054C169E170E08AE00E946A1E1092BE05C9
:103F5000209176058091C3059091C405A091C50577
:103F6000B091C605222311F0806801C08F7780933D
:103F7000C3059093C405A093C505B093C6050EEB89
:103F800015E0F80181918F010E944B1EF5E0073D7D
:103F90001F07B9F72FC161E270E08BE00E946A1E33
:103FA0008091AA048F3F39F08091AA0491E0980F84
:103FB0009093AA0402C08091AA040E944B1E10E0B4
:103FC000812F0E9437160E943C090E94591E1F5FD4
:103FD0001031B1F70FC161E070E08CE00E946A1E01
:103FE0008091D70505C161E070E085E60E946A1EF8
:103FF00089E2E816F10409F0FAC0D801EAE7F5E031
:104000008D91819385E0E33AF807D1F7E9C061E04B
:1040100070E086E60E946A1EEBE1EE16F10409F0FC
:10402000E6C0D801E3EAF5E08D91819385E0EE3BAF
:10403000F807D1F7D5C061E070E087E60E946A1EFC
:104040000E94730DCDC061E070E088E60E946A1E98
:1040500085E789838BE1E3EAF5E0DE0112960190C2
:104060000D928A95E1F76CE1CE0101960E940D0C4C
:104070000E948B0B83E08093770560E273E080E021
:1040800090E00E94BD2980917705843009F0AFC08F
:104090008FE70E94A9090E94BC098983853509F030
:1040A000A6C09EC061E070E08AE60E946A1E89E6B2
:1040B000898361E0CE0101960E940D0C0E948B0B5A
:1040C00083E08093770560E273E080E090E00E94F7
:1040D000BD2980917705843009F089C08FE70E945F
:1040E000A9090E94BC0989838E010E5F1F4F7E01C2
:1040F000EDE1EE0EF11C0E94BC09F80181938F01E5
:10410000EE15FF05C1F78BE1FE013296A3EAB5E09B
:1041100001900D928A95E1F78981893409F067C091
:104120005FC061E070E08BE60E946A1EF80180814A
:104130008093D8050E947C0D53C061E070E08CE64E
:104140000E946A1EF0E2EF16F10461F487E68983AB
:1041500080E2F801DE01129601900D928A95E1F756
:1041600061E203C087E4898361E0CE0101960E9489
:104170000D0C0E948B0B83E0809377056CE474E058
:1041800080E090E00E94BD2980917705843079F528
:104190008FE70E94A9090E94BC09873441F520C01D
:1041A00061E070E08DE60E946A1E89E1E816F10484
:1041B000F1F4D801EEEBF5E08D91819385E0E73DD8
:1041C000F807D1F70E94C1130BC061E070E08EE6E2
:1041D0000E946A1EF80180818093D7050E945D0DC0
:1041E00081E006C061E070E08AEC0E946A1E80E017
:1041F0000E944B1E0E94871EA196E6E00C945B2F46
:10420000A0E0B0E0E6E0F1E20C943D2FCAECD3E090
:1042100014E606E035E0F32E44E0E42E53E0D52E1C
:1042200062E0C62E86EE95E00E949A2C892B09F456
:104230009BC086EE95E00E94C72C282F8093350402
:104240004091340450E04730510560F7FA01EE52D6
:10425000FF4F0C946A2F853B29F781E0809334044B
:10426000E1CF823609F07DC0C0923404DBCF809369
:10427000330480933204D0923404D4CF9C0133278A
:104280003093310420933004909132049827909316
:104290003204E0923404C6CF382F222740913004F4
:1042A00050913104242B352B30933104209330046A
:1042B00090913204982790933204F092340425367A
:1042C000310508F4AFCF61E070E08CEC0E946A1E0B
:1042D00081E00E944B1E0E94871E43C020912E0445
:1042E00030912F04F901E653FC4F80839091320402
:1042F000982790933204C901019690932F048093DC
:104300002E0420913004309131048217930708F471
:1043100089CF0093340486CF8091320482130BC07E
:1043200060912E0470912F044AEC53E08091330485
:104330000E948E1E0DC062E070E08BEC0E946A1E2F
:10434000809133040E944B1E80916E050E944B1E8B
:10435000FE01812F11928A95E9F710922F04109295
:104360002E04109234045ECFCDB7DEB7E8E00C9493
:10437000592F81E080936F0580916F05882349F064
:1043800086EE95E00E949A2C892BB1F30E940021C1
:10439000F3CF0895AAE2B0E0E0EDF1E20C943B2FF8
:1043A0000E948E296B017C0181E00E94B00A86EE9A
:1043B00095E00E949A2C892B29F086EE95E00E94C8
:1043C000C72CF5CF4398299811E072E6B72EE9E2A1
:1043D000AE2E03E00E948E296C197D098E099F097B
:1043E000693C710581059105F0F11123E1F10E940D
:1043F0008E296B017C0185B1846285B980ED97E0DF
:104400000E94B607B982EAE7F5E0DE0112968A2D2E
:1044100001900D928A95E1F76AE2CE0101960E9421
:104420000D0C85B18B7D85B980E090E00E94B607C8
:10443000009377050E948B0B62E370E080E090E0D0
:104440000E94BD2980917705843061F4009377053F
:104450008FE70E94A9090E94BC0911E0823419F477
:1044600010E001C011E087E00E94B32A892BB1F46B
:1044700011E014C0439A299A85B1846285B986EE09
:1044800095E00E94C72C8D309105C1F074F40A9715
:10449000A9F04398299885B18B7D85B986EE95E082
:1044A0000E949A2C892B31F795CF8332910579F0B0
:1044B0008234910571F70E94B921EBCF62EB71E074
:1044C00086EE95E00E94742B0E94211EE2CF0E948E
:1044D000AA16DFCF8F929F92AF92BF92CF92DF92B8
:1044E000EF92FF921F93CF93DF9387E00E94B32A4E
:1044F000892B09F089C068EC70E080E090E00E94B0
:10450000BD2980E090E00E94B6070E948E294B01F1
:104510005C016B017C0180ECC80E82E1D81EE11CBD
:10452000F11C0E948E296C157D058E059F0530F4C7
:1045300087E00E94B32A892BA1F364C087E00E9420
:10454000B32A892B09F05EC080ED97E00E94B60780
:104550000E948E296B017C01D0E0C1E088E4880EC6
:1045600086E2981EA11CB11C11E087E00E94B32ACC
:10457000892B21F58C149D04AE04BF0430F480ED2A
:1045800097E00E94B607D1E0F0CF0E948E296C1907
:104590007D098E099F09693C71058105910528F304
:1045A0000E948E296B017C01C12719F080ED97E0F4
:1045B00002C080E090E00E94B607D7CF80E090E094
:1045C0000E94B607DD23B9F08091D70590E00196EF
:1045D00065E070E00E94DE2E8093D7050E945D0D9D
:1045E0000E94DC130E947C0D64EF71E080E090E09B
:1045F0000E94BD2909C080E00E94DF060E94F411DC
:104600000E94730D0E94CA21DF91CF911F91FF90EC
:10461000EF90DF90CF90BF90AF909F908F900895D4
:10462000CF92DF92EF92FF9280E00E940D080E94ED
:10463000E40761E081E10E94472A61E08DE00E9489
:10464000472A61E089E00E94472A61E08AE00E94EF
:10465000472A60E087E00E94472A60E08BE00E94E2
:10466000472A61E08BE00E94802A60E08CE00E9493
:10467000472A61E08CE00E94802A60E088E00E9486
:10468000472A61E088E00E94802A0E949F0740E05C
:1046900052EC61E070E086EE95E00E94E22D0E940F
:1046A000DC130E947C0D0E94C1138FEF8093AA043B
:1046B0000E94F90778940E948E296B017C018091F9
:1046C000AA048F3F59F40E948E296C197D098E0926
:1046D0009F09603D77408105910588F380ED97E063
:1046E0000E94B60761E087E00E94802A439A299AD7
:1046F00086EE95E00E949A2C892B29F086EE95E0B3
:104700000E94C72CF5CF6DEF72E086EE95E00E9417
:10471000552B88E893E00E94620C64E173E086EE1A
:1047200095E00E94552B4AE050E063E070E086EE91
:1047300095E00E94252C62E370E080E090E00E940A
:10474000BD2986EE95E00E949A2C04970CF186EE26
:1047500095E00E94C72C82349105D1F486EE95E055
:104760000E94C72C8E34910599F486EE95E00E9444
:10477000C72C8434910561F486EE95E00E94C72C25
:10478000819731F480E090E00E94B6070E94CA2130
:1047900040917B0550917C0560917D0570917E056F
:1047A000DB01CA010197A109B1090497A105B1056F
:1047B00068F44093A904433029F440EA56E861E0E4
:1047C00070E004C040E052EC61E070E086EE95E0FD
:1047D0000E94E22D0E946A224398299880E090E08E
:1047E0000E94B6070E94C1131092C9048091C305AC
:1047F00083FF11C080918F05882351F08091960529
:10480000882331F080919D05882311F087E001C055
:1048100085E08093C90480E00E94B00A8091CA04B8
:104820000E94E4090E948B0B10923F0410923E04F8
:1048300010923D04F12C8091D8058F15B0F062E301
:1048400070E080E090E00E94BD2980ED97E00E943A
:10485000B60762E370E080E090E00E94BD2980E04E
:1048600090E00E94B607F394E6CF8091A20584FF02
:1048700008C0982F987181E0983109F080E00E947B
:10488000B0118FE00E940D08FF90EF90DF90CF9065
:104890000895EF92FF920F931F93CF93DF938C01B4
:1048A0006EE770E086EE95E00E945906E801F12C73
:1048B000F0E2EF2E8E0188818D57823048F46DE74B
:1048C00070E086EE95E00E94590688818E258883E7
:1048D0002196F801608186EE95E00E94F42CF39415
:1048E000F9E0FF12E7CF6EE770E086EE95E00E94F8
:1048F0005906CDB7DEB7E6E00C945B2FA9E0B0E037
:10490000E4E8F4E20C94432F9091CB0491110EC093
:104910009EEF99838A836B8350E0559547954C832E
:104920002D83198618861F821E822EC04091D004C6
:10493000842F90E0B4E095958795BA95E1F7242F00
:104940002F7030E08217930719F18DEF89831B8256
:10495000FE01349650E0842F90E0A4E09595879571
:10496000AA95E1F7242F2F7030E08217930749F0C2
:10497000DC01AF52BB4F8C918193405F5F5F56303B
:1049800051F74093D0045A83CE0101960E944924E6
:104990008091CB0490E0019666E070E00E94DE2EEC
:1049A0008093CB042996E2E00C945F2FA0E0B0E066
:1049B000ECEDF4E20C943C2F6C016EE770E086EEB7
:1049C00095E00E9459068601E12CF12CC0E0D0E070
:1049D00030E2B32EF801608183E8860F823078F4EC
:1049E0006DE770E086EE95E00E945906F80160815F
:1049F0006B2570E086EE95E00E94590604C086EEB5
:104A000095E00E94F42CE114F10459F0F801808142
:104A10009E01280F311DC901C92FDD27C80FD91FDD
:104A2000DD273FEFE31AF30A89E0E816F10459F0B5
:104A300028E0E216F10421F48C2F8095F60180879E
:104A40000F5F1F4FC7CFCDB7DEB7E9E00C94582FEB
:104A5000A9E0B0E0EEE2F5E20C94432FE82F362F08
:104A60008091CB0490E0019664E270E00E94DE2E1B
:104A70008093CB0458E9598350E15A83813089F0FF
:104A800048F08230B9F08330D9F48B8381EF8C8386
:104A90003D8319C085E08B8381EF8C832F5F2D834D
:104AA00012C08B8381EF8C8384E6489FA001112480
:104AB0005D8309C084E08B8381EF8C83ED8303C029
:104AC0000E94ED1104C0CE0101960E94D6242996C1
:104AD000E2E00C945F2FA2E0B0E0E1E7F5E20C9495
:104AE000382F182F762E2A8349830E949A296B012A
:104AF0007C018091E1048090CC049090CD04A09042
:104B0000CE04B090CF042A8149818823C1F0D70117
:104B1000C60188199909AA09BB094C015D0191EEEA
:104B200089169EE29906A104B10420F1241708F425
:104B3000422F202F672D812F0E94282513C0D701D7
:104B4000C60188199909AA09BB094C015D0191E3C5
:104B5000891695E79906A104B10460F0672D812FAD
:104B60000E947E24C092CC04D092CD04E092CE0468
:104B7000F092CF042296EDE00C94542FA2E2B0E024
:104B8000E4ECF5E20C94392F8CE00E94CB09811102
:104B90000FC06CE173E086EE95E00E94862B439A8D
:104BA000299A80E00E94B00A0E948B0B43982998B2
:104BB00086EE95E00E949A2C892B01F186EE95E015
:104BC0000E94C72C9091A904992319F00E941814EF
:104BD000EFCF40913E0450E09A012F5F3F4F2F717D
:104BE000332760913F0470E02617370709F3FA0175
:104BF000E75BFB4F808320933E04DACF80917705FB
:104C0000843009F086C00E949A29611571058105DA
:104C1000910549F06093BB047093BC048093BD047C
:104C20009093BE040CC081E090E0A0E0B0E08093DF
:104C3000BB049093BC04A093BD04B093BE048091C8
:104C4000AD049091AE0481609093AE048093AD0466
:104C500083E0809377058FE70E94A90909E614E0B5
:104C60000E94BC09F80181938F01F4E002371F070D
:104C7000B9F72091720480916904982F922796FFCA
:104C80003BC090E4922790937204982F98739833C6
:104C9000F1F410E0212F30E080916904877090E0FA
:104CA000821793074CF11F5F2091A205812F90E09E
:104CB000FC01E759FB4F24FF04C080810E94CF1103
:104CC000E9CF608186EE95E00E94F42CE3CF8F73EC
:104CD00099F480916A048093B60480916B04809368
:104CE000B40480916C048093B30480916F0490E0CD
:104CF0009093AC048093AB0480913D04813019F40F
:104D000082E080933D0480913D04833011F4109241
:104D10003D040E949A296B017C018091AF0490911F
:104D2000B004A091B104B091B2040097A105B105FF
:104D3000C9F0A7019601281B390B4A0B5B0BDA015E
:104D4000C901883B9B40A105B10560F00E94FA09AA
:104D50008093B5041092AF041092B0041092B10485
:104D60001092B2048091BF049091C004A091C1043C
:104D7000B091C20446015701881A990AAA0ABB0ACF
:104D80008AE795E00E94270886169706A806B906C6
:104D900008F4B3C0C092BF04D092C004E092C10432
:104DA000F092C2040E9457068091AA048830A0F0B5
:104DB0008091C3059091C405A091C505B091C60529
:104DC0005CE1B695A795979587955A95D1F7892B6C
:104DD0008A2B8B2B09F0CCC18091AA048F5F809322
:104DE000AA048091BB049091BC04A091BD04B09131
:104DF000BE040097A105B105F1F0C81AD90AEA0A64
:104E0000FB0A8AE795E00E9427086C157D058E0550
:104E10009F0508F01FC18091C30584FD04C080ED8B
:104E200097E00E94B6071092BB041092BC04109247
:104E3000BD041092BE0490917204907C9093720411
:104E400050913E0480913F0420913D04581709F48D
:104E50001EC1223009F01BC1905890937204E0915A
:104E6000A205E770F0E0E658FC4F6081693008F079
:104E7000F6C0615040E04613F4C080933F0487E3DE
:104E8000840F90917204892B8093720440934004A4
:104E900083E080933D0485B1846285B910918705D4
:104EA0008091C904811142C18091C30582FD4AC12C
:104EB000812F0E94AB0A8091CA040E94E409E0910C
:104EC000A205E770F0E0E658FC4F608182E794E0CD
:104ED0000E94C60B8091C30582FD3EC1E091CA04C9
:104EE000EF5FE093CA04E83109F43FC1F0E0E6580F
:104EF000FA4F8785882309F438C10E94350C813028
:104F000069F58091A205887149F18091AD04909175
:104F1000AE04880F991F9093AE048093AD0483E094
:104F2000809377050E948B0B0E949A296093AF04AF
:104F30007093B0048093B1049093B204672B682BF4
:104F4000692B61F481E090E0A0E0B0E08093AF04D1
:104F50009093B004A093B104B093B2048091A205E1
:104F600084FF2BC08091BB049091BC04A091BD0430
:104F7000B091BE04892B8A2B8B2BF9F08091AD0464
:104F80009091AE048E7F0E945D09182F6091AB0452
:104F90008091B6040E940E14482F612F8091B504B1
:104FA00049A30E940E140091D805282F49A16091B1
:104FB000B3048091B4040E946B2585B18B7D85B9C3
:104FC0008091C7048130C1F018F08230B1F1DEC0A9
:104FD00087E00E94B32A892B09F0D8C081E0809332
:104FE000C7040E948E296093C3047093C404809305
:104FF000C5049093C604CAC087E00E94B32A892BD7
:1050000031F50E948E29C090C304D090C404E09072
:10501000C504F090C6046C197D098E099F09693E8C
:1050200073408105910508F4B1C082E08093C70404
:1050300080ED97E00E94B607A9C087E00E94B32ADE
:10504000892B09F4A3C080E090E00E94B60710927B
:10505000C7049CC080E090E00E94B607ECCE68E0F8
:1050600009CF851709F409CF4F5F242F30E090E076
:10507000F901EE58FB4FDC01A75BBB4F7C917083BD
:10508000F901E05CFB4F708301968F71F4CE243000
:10509000B1F42091400481E494E0A3E7B4E0FC0182
:1050A0003E2F381B321718F431913D93F9CF87E327
:1050B000820F90917204892B80937204E9CE8091C3
:1050C000C704823059F4916090937204439A299AEC
:1050D0008E010F5F1F4FF12CB80111C04398299822
:1050E00080913D04811103C081E080933D04809153
:1050F0003D04833069F784E080933D04E9CF8F2D30
:1051000069A37AA30E943716F801819391938F01C6
:10511000F39469A17AA1F0E1FF12F1CF8091A20589
:1051200043E754E087700E94AC08B5CE112309F420
:10513000BBCE9091C80421E0290F2093C804981396
:10514000B3CE20C08BE00E94B32A892B09F0B0CEE9
:10515000439A299A17E0ACCE8BE00E94B32A892BA0
:1051600009F0BCCE43982998B9CE1092CA04C5CE96
:105170008091AA04883011F4439A299A89E0809397
:10518000AA04BBCE1092C80411508ECEA296ECE0B9
:105190000C94552F8230E8F4E82FF0E0EE0FFF1F5B
:1051A000E752FA4F71836083813041F0809169004A
:1051B0008C7F842B80936900E89A08958091690020
:1051C000440F551F440F551F837F842B8093690024
:1051D000E99A08951F920F920FB60F9211242F9300
:1051E0003F934F935F936F937F938F939F93AF936F
:1051F000BF93EF93FF938091D9059091DA05892BA6
:1052000029F0E091D905F091DA050995FF91EF9128
:10521000BF91AF919F918F917F916F915F914F91CE
:105220003F912F910F900FBE0F901F9018951F92D6
:105230000F920FB60F9211242F933F934F935F93CA
:105240006F937F938F939F93AF93BF93EF93FF934E
:105250008091DB059091DC05892B29F0E091DB053D
:10526000F091DC050995FF91EF91BF91AF919F916E
:105270008F917F916F915F914F913F912F910F90FF
:105280000FBE0F901F9018951F920F920FB60F929E
:1052900011242F933F938F939F93AF93BF9380914C
:1052A000DE059091DF05A091E005B091E105309118
:1052B000DD0523E0230F2D3720F40196A11DB11D3C
:1052C00005C026E8230F0296A11DB11D2093DD0520
:1052D0008093DE059093DF05A093E005B093E10590
:1052E0008091E2059091E305A091E405B091E50578
:1052F0000196A11DB11D8093E2059093E305A09353
:10530000E405B093E505BF91AF919F918F913F91D7
:105310002F910F900FBE0F901F9018952FB7F894F4
:105320006091DE057091DF058091E0059091E105C7
:105330002FBF08953FB7F8948091E2059091E3055F
:10534000A091E405B091E50526B5A89B05C02F3FC7
:1053500019F00196A11DB11D3FBF6627782F892F37
:105360009A2F620F711D811D911D42E0660F771FFC
:10537000881F991F4A95D1F70895CF92DF92EF9237
:10538000FF92CF93DF936B017C010E949A29EB017E
:10539000C114D104E104F10479F00E949A296C1B34
:1053A0007D0B683E7340A0F381E0C81AD108E10884
:1053B000F108C851DC4FECCFDF91CF91FF90EF9017
:1053C000DF90CF900895789484B5826084BD84B5D1
:1053D000816084BD85B5826085BD85B5816085BDF0
:1053E000EEE6F0E0808181608083E1E8F0E0108209
:1053F000808182608083808181608083E0E8F0E04A
:10540000808181608083E1EBF0E080818460808333
:10541000E0EBF0E0808181608083EAE7F0E080816A
:1054200084608083808182608083808181608083CA
:105430008081806880831092C1000895833081F05C
:1054400028F4813099F08230A1F008958630A9F0D7
:105450008730B9F08430D1F4809180008F7D03C013
:10546000809180008F7780938000089584B58F7736
:1054700002C084B58F7D84BD08958091B0008F7780
:1054800003C08091B0008F7D8093B0000895CF93CA
:10549000DF9390E0FC01ED50F44F2491FC01E95FB3
:1054A000F34F8491882349F190E0880F991FFC0104
:1054B000E15DF34FA591B4918B5D934FFC01C591D4
:1054C000D4919FB7611108C0F8948C9120958223E4
:1054D0008C93888182230AC0623051F4F8948C91B5
:1054E000322F309583238C938881822B888304C04C
:1054F000F8948C91822B8C939FBFDF91CF9108956C
:10550000A1E0B0E0E6E8FAE20C94412F282F30E069
:10551000F901E152F44F8491F901ED50F44F1491E7
:10552000F901E95FF34F04910023C9F0882321F0CA
:1055300069830E941E2A6981E02FF0E0EE0FFF1FB1
:10554000EB5DF34FA591B4919FB7F8948C916111E5
:1055500003C01095812301C0812B8C939FBF21969E
:10556000E4E00C945D2FCF93DF93282F30E0F90116
:10557000E152F44F8491F901ED50F44FD491F901C7
:10558000E95FF34FC491CC2391F081110E941E2A50
:10559000EC2FF0E0EE0FFF1FE55EF34FA591B49105
:1055A0002C912D2381E090E021F480E002C080E086
:1055B00090E0DF91CF9108958E3008F08E50877083
:1055C00020919D0190E4299F90011124822B8093CA
:1055D0007C0080917A00806480937A0080917A00C8
:1055E00086FDFCCF809178002091790090E0922B8D
:1055F0000895A0E0B0E0EFEFFAE20C943D2F6C01CB
:105600007A01EB01E60EF71E00E010E0CE15DF0593
:1056100061F06991D601ED91FC910190F081E02D4E
:10562000C6010995080F191FF1CFC801CDB7DEB724
:10563000E8E00C94592F6115710589F0DB010D909C
:105640000020E9F7AD0141505109461B570BDC0121
:10565000ED91FC910280F381E02D0995089580E0A1
:1056600090E00895EF92FF920F931F93CF93DF93F3
:105670008C01FB01C0E0D0E064917F018FEFE81A5C
:10568000F80A662361F0D801ED91FC910190F08158
:10569000E02DC8010995C80FD91FF701EDCFCE0144
:1056A000CDB7DEB7E6E00C945B2F0E941B2B08956C
:1056B000DC01ED91FC910190F081E02D09950895B8
:1056C0000F931F93CF93DF93EC016DE00E94582B53
:1056D0008C016AE0CE010E94582B800F911FDF9150
:1056E000CF911F910F9108950F931F93CF93DF9345
:1056F000EC010E94322B8C01CE010E94602B800FA6
:10570000911FDF91CF911F910F9108950F931F93D8
:10571000CF93DF93EC010E941B2B8C01CE010E94E2
:10572000602B800F911FDF91CF911F910F910895F2
:105730000F931F93CF93DF93EC010E94582B8C01A2
:10574000CE010E94602B800F911FDF91CF911F919E
:105750000F910895A1E2B0E0E0EBFBE20C94392F49
:105760007C01C42EE52FCB01D22E19A221E02D15EC
:1057700010F02AE0D22E8E010F5D1F4F8D2C912C40
:10578000A12CB12C6C2D7E2FA50194010E94F22E2C
:105790008C2DD29E80191124015011098A3010F4E9
:1057A000805D01C0895CF8018083211531054105C8
:1057B000510521F0C22EE32FCA01E4CFB801C70181
:1057C0000E941B2BA196ECE00C94552FA0E0B0E0BA
:1057D000ECEEFBE20C943D2FEC016A017B012115FC
:1057E000310541F4E881F9810190F081E02D642FC9
:1057F00009951DC02A303105A9F477FF12C06DE26A
:105800000E94582B8C0144275527BA014C195D0979
:105810006E097F092AE0CE010E94AA2B800F911FFA
:1058200006C02AE0B701A601CE010E94AA2BCDB77F
:10583000DEB7E8E00C94592F9A01AB01662757FDBB
:105840006095762F0E94E62B08950F931F93CF93B8
:10585000DF93EC019A01AB01662757FD6095762F27
:105860000E94E62B8C01CE010E94602B800F911FBD
:10587000DF91CF911F910F9108952115310549F4C2
:10588000DC01ED91FC910190F081E02D642F0995F0
:1058900008950E94AA2B08959A01462F50E060E0D7
:1058A00070E00E943D2C08959A01AB0160E070E029
:1058B0000E943D2C08950F931F93CF93DF93EC012B
:1058C0000E943D2C8C01CE010E94602B800F911F05
:1058D000DF91CF911F910F9108950F931F93CF9355
:1058E000DF93EC019A01AB0160E070E00E943D2C77
:1058F0008C01CE010E94602B800F911FDF91CF9110
:105900001F910F9108950F931F93CF93DF93EC0195
:105910009A01462F50E060E070E00E943D2C8C011F
:10592000CE010E94602B800F911FDF91CF911F91BC
:105930000F910895FC0124853585F901E05CFF4F46
:1059400080819181F901EE5BFF4F20813181821BC3
:10595000930B8F7399270895FC0184859585FC012D
:10596000E05CFF4F40815181FC01EE5BFF4F2081E5
:1059700031814217530741F00190F081E02DE80F8B
:10598000F91F808190E008958FEF9FEF0895FC014B
:1059900084859585FC01E05CFF4F40815181FC01CD
:1059A000EE5BFF4F208131814217530779F0A081D0
:1059B000B181A80FB91F8C91208131812F5F3F4F9A
:1059C0002F7333273183208390E008958FEF9FEF6B
:1059D0000895FC0181A1882329F0A489B5898C91BF
:1059E00086FFFBCF11A20895CF93DF93FC0126859C
:1059F0003785D901A05CBF4F8D919C91119701967D
:105A00008F739927E901CE5BDF4F48815981841755
:105A10009507D9F30D90BC91A02DA20FB31F6C93E5
:105A2000A685B785A05CBF4F11969C938E93A689DF
:105A3000B7892C9181E090E0078C02C0880F991FF4
:105A40000A94E2F7282B2C9381E081A30488F5893E
:105A5000E02D80818064808381E090E0DF91CF91B0
:105A6000089508951F920F920FB60F9211242F934D
:105A70003F934F938F939F93EF93FF938091C00039
:105A800082FD1CC04091C60080918C0690918D06CD
:105A900001968F73992720918E0630918F06821779
:105AA000930771F0E0918C06F0918D06E45BF94F5D
:105AB000408390938D0680938C0602C08091C6002F
:105AC000FF91EF919F918F914F913F912F910F9067
:105AD0000FBE0F901F90189586EE95E00E949A2CAD
:105AE000892B11F00E94312D08951F920F920FB64D
:105AF0000F9211242F933F938F939F93EF93FF93D4
:105B0000209148063091490680914A0690914B06B3
:105B10002817390731F48091C1008F7D8093C1002F
:105B200014C0E0914A06F0914B06E85FF94F2081DE
:105B300080914A0690914B0601968F739927909316
:105B40004B0680934A062093C600FF91EF919F91E8
:105B50008F913F912F910F900FBE0F901F9018952E
:105B6000A0E0B0E0E6EBFDE20C94392FFC011382DB
:105B7000128288EE93E0A0E0B0E084839583A68350
:105B8000B7838CEB93E09183808375876487578715
:105B90004687318B208B138B028BF58AE48AD78A58
:105BA000C68AB18EA08E938E828E8F85848F8889CF
:105BB000858F8989868F8A89878F8B8980A3ECE07E
:105BC0000C94552FCF92DF92EF92FF92CF93DF93F9
:105BD000EC016A017B01411581EE580761057105F1
:105BE000F9F0EC89FD8981E090E008A002C0880FFF
:105BF000991F0A94E2F7808360E079E08DE390E0FA
:105C0000A70196010E94F22E215031094109510944
:105C10005695479537952795211580E1380798F0D7
:105C2000EC89FD89108260E874E88EE190E0A701BC
:105C300096010E94F22E21503109410951095695D1
:105C4000479537952795E889F9893083EA89FB8953
:105C5000208319A2EE89FF89408181E090E09C01B8
:105C60000C8C02C0220F331F0A94E2F7422B4083B0
:105C7000EE89FF8940819C010D8C02C0220F331FE9
:105C80000A94E2F7422B4083EE89FF8940819C0110
:105C90000E8C02C0220F331F0A94E2F7422B40837E
:105CA000EE89FF8920810F8C02C0880F991F0A940A
:105CB000E2F7809582238083DF91CF91FF90EF9070
:105CC000DF90CF9008958F929F92AF92BF92CF9224
:105CD000DF92EF92FF920F931F9381E08F9385E005
:105CE0008F9387E08F9383E08F9384E08F93E6EC2C
:105CF0008E2E912CF2ECAF2EB12CA1ECCA2ED12C11
:105D0000B0ECEB2EF12C04EC10E025EC30E048E098
:105D100056E06CE476E086EE95E00E94B02D0F90A0
:105D20000F900F900F900F901F910F91FF90EF9099
:105D3000DF90CF90BF90AF909F908F9008950E947A
:105D4000E3290E941023CCE6DDE20E94BE252097C5
:105D5000E1F30E946C2DF9CFA29FB001B39FC00167
:105D6000A39F700D811D1124911DB29F700D811D87
:105D70001124911D08950E94AC2EA59F900DB49FF3
:105D8000900DA49F800D911D11240895B7FF0C94D0
:105D9000BB2E0E94BB2E821B930B0895DB018F93B9
:105DA0009F930E94BB2EBF91AF91A29F800D911D2A
:105DB000A39F900DB29F900D1124089597FB072E7D
:105DC00016F4009407D077FD09D00E94702F07FCCD
:105DD00005D03EF4909581959F4F089570956195FB
:105DE0007F4F0895A1E21A2EAA1BBB1BFD010DC017
:105DF000AA1FBB1FEE1FFF1FA217B307E407F5077B
:105E000020F0A21BB30BE40BF50B661F771F881F56
:105E1000991F1A9469F760957095809590959B01EC
:105E2000AC01BD01CF010895052E97FB1EF400942F
:105E30000E942B2F57FD07D00E94F22E07FC03D0A3
:105E40004EF40C942B2F50954095309521953F4F53
:105E50004F4F5F4F089590958095709561957F4F56
:105E60008F4F9F4F08952F923F924F925F926F9264
:105E70007F928F929F92AF92BF92CF92DF92EF92DA
:105E8000FF920F931F93CF93DF93CDB7DEB7CA1B5B
:105E9000DB0B0FB6F894DEBF0FBECDBF09942A8886
:105EA000398848885F846E847D848C849B84AA842E
:105EB000B984C884DF80EE80FD800C811B81AA81BB
:105EC000B981CE0FD11D0FB6F894DEBF0FBECDBF86
:105ED000ED010895EE0FFF1F0590F491E02D099458
:105EE000AA1BBB1B51E107C0AA1FBB1FA617B70700
:105EF00010F0A61BB70B881F991F5A95A9F780951C
:105F00009095BC01CD0108958F929F92AF92BF9260
:105F1000CF92DF92EF92FF92CF93DF93EC016881F3
:105F200079818A819B81611571058105910521F433
:105F300064E279ED8BE597E02DE133EF41E050E04D
:105F40000E94142F49015A019B01AC01A7EAB1E458
:105F50000E94BB2E6B017C01ACEEB4EFA501940155
:105F60000E94C92EC60ED71EE81EF91EF7FE06C0F7
:105F700081E0C81AD108E10880E8F80AC882D9820D
:105F8000EA82FB82C701B6019F77DF91CF91FF9034
:105F9000EF90DF90CF90BF90AF909F908F9008953B
:105FA0000E94842F089586E091E00E94842F089536
:105FB0006093060170930701809308019093090193
:105FC00008952F923F925F926F927F928F929F924D
:105FD000AF92BF92CF92DF92EF92FF920F931F93F7
:105FE000CF93DF938B01EA016115710521F0DB018D
:105FF0008C9311969C93209739F09E012250310981
:106000002332310508F0D8C07C016701BFEFCB1AFD
:10601000DB0A5601F7016080862D90E00E94133163
:10602000892B11F07601F1CFFDE26F120AC0570102
:1060300082E0A80EB11CD70111966C90772473945E
:106040000BC0BBE26B1207C05701E2E0AE0EB11C01
:10605000D70111966C90712CCE018F7E892B89F41B
:10606000B0E36B1237C0F50180818F7D8835D1F4A4
:106070006180F2E0AF0EB11C872D8260782EC0E106
:10608000D0E0CA30D10551F1C031D10521F0C8307E
:10609000D10599F409C0CC24CA94DC2CEC2CAFE0D7
:1060A000FA2E22C0209769F7C8E0D0E0CC24CA9429
:1060B000DC2CEC2CFFE1FF2E17C06FEF7FEFCB0144
:1060C0009E01442737FD4095542F0E94F22E69010E
:1060D0007A010AC02097A9F6CAE0D0E0E9E9CE2EFD
:1060E000DC2CEC2CE9E1FE2EF50160E020E030E054
:1060F000A9014E01AA2497FCA094BA2C1F0170EDAF
:10610000572E560CA9E0A51570F48FEB860D8A3139
:1061100018F499EC592E06C08FE9860D8A3148F59E
:1061200089EA582E560C852D90E08C179D070CF5AA
:106130006F3FD9F0C216D306E406F50698F0C50104
:10614000B4010E94CE2E9B01AC01852D90E0A0E011
:10615000B0E0280F391F4A1F5B1F281739074A076D
:106160005B0710F46FEF01C061E03196D1016C90D4
:10617000C5CF0115110551F0662311F0319703C009
:1061800071FE04C03297D801ED93FC9370FE07C0F6
:1061900050954095309521953F4F4F4F5F4F67FF8A
:1061A00010C082E290E090939106809390066FEF8A
:1061B0007FEF8FEF9FEF07C060E070E080E090E03E
:1061C00002C0B901CA01DF91CF911F910F91FF90D9
:1061D000EF90DF90CF90BF90AF909F908F907F9087
:1061E0006F905F903F902F900895FC01882799272A
:1061F000E89421912032E9F3293010F02E30C8F3D1
:106200002B3241F02D3239F4689404C00E9447319A
:10621000820F911D219120532A30C0F31EF49095D6
:1062200081959F4F0895911150C0803219F0895087
:106230008550D0F7089548EC53E00E94203108952E
:10624000FA01A191B081009719F41097E1F0CD0106
:10625000DC01CD010D90002011F4C00113C0FB0141
:106260002191222319F02015D9F7F3CFFB012191B9
:10627000201519F41E92119606C02223C1F70D9025
:106280000020A1F7D001FA01A193B08308957AE02C
:10629000979F902D879F802D910D11240895F99936
:1062A000FECF92BD81BDF89A992780B50895262F1B
:1062B000F999FECF1FBA92BD81BD20BD0FB6F894EB
:1062C000FA9AF99A0FBE019608959927882708959A
:0462D000F894FFCF70
:1062D40000009206200001000000FF0002000200FE
:1062E400020002000200020002000200020002009A
:1062F40002000200020002000200028025000005E4
:10630400400AA1204EA50020244EA52C2330C01203
:1063140000001A400AA1204EA5001B1E27522C2360
:10632400308025000005400AA1204EA50020244EFF
:10633400A52C2330004B000006400AD0009D4900E4
:106344007B289D492C233000E1000005400A4501CB
:10635400D7DC03B81E0EBF00232E48E801008A4094
:106364000A6001555502AD1E20000023C80154588F
:106374002074696D656F75742100596573004E6FE3
:10638400002C00386368004E2F41002C205B005D18
:106394002028002900486F70206368616E6E656C68
:1063A400200020402000456E746572696E6720618C
:1063B40064617074697665206368616E6E656C20D3
:1063C40073656C656374696F6E2C207069636B69A7
:1063D4006E673A007363616E6E6572206D6F6465FB
:1063E400004E4F5420454E41424C45440053656E87
:1063F40064696E672073657474696E677320746F63
:106404002052580A00526573657474696E6720736C
:10641400657474696E6773206F6E2052580A004168
:10642400626F727465642065646974730A00696ECE
:1064340076616C69642073656C656374696F6E0062
:106444000D0A496E76616C696420696E70757420FA
:106454002D20646973636172646564210700536568
:106464007474696E677320736176656420746F2039
:10647400454550524F4D0A00526576657274656405
:106484002073657474696E67732066726F6D20453E
:106494004550524F4D0A004C6F616465642066613B
:1064A40063746F72792064656661756C74730A0035
:1064B4004B657920616E64206368616E6E656C73F0
:1064C4002072616E646F6D697A65640A004F70654D
:1064D4006E4C52536E672054582073746172746901
:1064E4006E672000206F6E20485720006D6F647522
:1064F4006C65206C6F636B65643F00342B3400382B
:1065040000382B340031320031322B340031360064
:1065140050504D0052535349005344410053434C8F
:1065240000525844005458440041494E004C4245DE
:1065340045500053504B54524D0053425553005351
:10654400554D44004C4C494E440000070B0C1011AF
:106554001500B7012B032F033103350338033D0323
:10656400B7014003440349034D0351035503590341
:106574005D0363036A036F0374038D028D028D024E
:106584008D02160A1322312900000000F42CF92A86
:086594009A2CC72CAC2CE92C59
:107E00000F92CDB7DEB7112484B714BE81FFF1D035
:107E100082E08093C00088E18093C10086E0809377
:107E2000C20080E18093C4008EE0CDD088249924E4
:107E3000CC24C394F5E0DF2EE1E1EE2E73E0F72EC3
:107E4000B6D0082F813479F4B2D08983C2D0898129
:107E5000823811F481E005C0813811F485E001C059
:107E600083E09ED09AC0823411F484E103C085344B
:107E700019F485E0B6D091C0853561F498D0082F0B
:107E800010E095D090E0982E8824802A912A880CC2
:107E9000991C82C0863521F484E0A3D080E0E1CF34
:107EA000843609F04CC083D082D0A82E80D0B82E62
:107EB00000E011E07CD0F80181938F01AE16D1F77C
:107EC00088D0FB2DF53489F4E0E0F1E00BC0F9999E
:107ED000FECF92BC81BC0894811C911C819180BD15
:107EE000FA9AF99AEA1598F358C08B2D863409F05E
:107EF00054C0F401F7BEE89507B600FCFDCFF401CD
:107F0000A0E0B1E02C9130E011968C91119790E0B7
:107F1000982F8827822B932B12960C01C7BEE895C9
:107F20001124329681E0A038B80761F7F401D7BE7A
:107F3000E89507B600FCFDCFE7BEE8952EC0843774
:107F4000F1F435D034D0182F32D0B82E42D0FB2DDA
:107F5000F63421F4F40105914F010CC0FB2DF534EA
:107F600049F4F999FECF92BC81BC0894811C911C04
:107F7000F89A00B5802F14D0115049F70EC08537FC
:107F800039F427D08EE10CD085E90AD08FE069CF93
:107F9000813511F488E017D01CD080E101D050CF9A
:107FA0009091C00095FFFCCF8093C600089580910A
:107FB000C00087FFFCCF8091C00084FD01C0A89560
:107FC0008091C6000895E0E6F0E098E19083808318
:107FD0000895EDDF803219F088E0F5DFFFCF84E10E
:107FE000DFCF1F93182FE3DF1150E9F7F2DF1F9166
:0E7FF0000895282E80E0E7DFEE27FF27099492
:027FFE0001057B
:0400000300007E007B
:00000001FF
